:1075D400758400852ED2852FD3E4F52FF52E30380F
:1075E40010E50D852DF0A4252EF52EE5F0352FF5AB
:1075F4002F22907610303E0312760022E50E251BD2
:10760400F50EE51F351AF51F93F50D227F82858847
:107614008C8F9295989B9EA1A4A7AAADB0B3B6B93E
:10762400BBBEC1C3C6C9CBCED0D3D5D7D9DCDEE06F
:10763400E2E4E6E7E9EBEDEEF0F1F2F4F5F6F7F863
:10764400F9FAFBFCFCFDFDFEFEFEFEFEFEFEFEFE68
:10765400FEFDFDFCFCFBFAFAF9F8F7F6F4F3F2F0A0
:10766400EFEDECEAE8E7E5E3E1DFDDDBD8D6D4D102
:10767400CFCDCAC8C5C2C0BDBAB7B4B2AFACA9A653
:10768400A3A09D9A9794908D8A8784817E7A77743B
:10769400716E6B6865625F5C595653504D4A47443E
:1076A400423F3C393734322F2D2A282624211F1DEE
:1076B4001B1918161412110F0E0C0B0A08070605D5
:1076C40004040302020101000000000000000000A5
:1076D4000001010202030405060708090A0B0D0E46
:1076E4001011131516181A1C1E20222427292B2EBC
:1076F400303335383A3D404245484B4E5154565943
:0C7704005C606366696C6F7275787B7F57
:107DF000D2F4C2F5C2F675840F85F0C8127A1674F3
:107E000003127E3F127A067403127E3F1279F51236
:107E100079F57403127E3F1279F57402127E3F12D7
:107E200079F57428127EAB7406127EAB740E127E46
:107E3000AB7401127EAB127A067480127EAB22C044
:107E400000A2E092F3A2E192F2A2E292F1A2E39206
:107E5000F0D2F475840F85F0C8C2F47830D8FE856E
:107E6000F0C87830D8FED00022C00075840FA2E49C
:107E700092F3A2E592F2A2E692F1A2E792F0D2F496
:107E800085F0C8C2F47830D8FE85F0C87830D8FEC6
:107E9000D00022EF75840FD2F5C2F685F0C8127EAD
:107EA000691279F5127E3F1279F52275840FC2F5B9
:107EB000C2F685F0C8127E691279F5127E3F1279FA
:107EC000F522EF14A2E492E6C2E4D2E7127EAB22DE
:107ED000740F127EAB22740D127EAB227F01127ED4
:107EE000C278107F20127E93D8F9227F11127EC2B1
:0A7EF00078107F20127E93D8F9224B
:10749700C293758400D2C2C2C6D2C6C2C4D2C5C204
:1074A700C330C3FD74A0F5C2C2C5C2C330C3FD8ECD
:1074B700C2C2C330C3FD8FC2C2C330C3FD8DC2C2B7
:1074C700C330C3FDD2C4C2C320C4FD127A06D2930F
:1074D70022758400C2C3D2C530C3FD74A0F5C2C2F1
:1074E700C5C2C330C3FD8EC2C2C330C3FD8FC2C283
:1074F700C330C3FDC2C4D2C5C2C330C3FD74A1F536
:10750700C2C2C5C2C330C3FDC2C2C2C330C3FD8538
:10751700C207D2C4C2C320C4FD22D2C2C2C6D2C6C9
:10752700D2C4C2C320C4FD22C293758400D2C2C292
:10753700C6D2C6C2C4D2C5C2C330C3FD74A0F5C289
:10754700C2C5C2C330C3FD8EC2C2C330C3FD8FC222
:10755700C2C330C3FD8C838D827B80E0A3F5C2C29A
:10756700C330C3FDDBF5D2C4C2C320C4FD127A0603
:10757700D29322758400C2C3D2C530C3FD74A0F56F
:10758700C2C2C5C2C330C3FD8EC2C2C330C3FD8FE2
:10759700C2C2C330C3FDC2C4D2C5C2C330C3FD74A7
:1075A700A1F5C2C2C5C2C330C3FD8C838D82C2C3DD
:1075B70030C3FDE5C2F0A31BBB01F3C2C2C2C33097
:0D75C700C3FDE5C2F0D2C4C2C320C4FD2242
:030003000259643B
:01000B0032C2
:0300130002771061
:1065BB0075FF0775FFDE75FFAD75840F75E1077508
:1065CB00E21475E34475840F75A43575A50975A69A
:1065DB00BB75A7FF759CFF759D00759EF0759FF8A9
:1065EB0075D8FF75E8FF75F80F75AD0F75840175DC
:1065FB00893075888F75840275893075888F75849D
:10660B000F758A80758C67780874FF000000000096
:10661B0000000000000000D5E0F1D8EDE58C30E77C
:10662B00FB759701758A0043890475840075B71053
:10663B0075840F438901758D02758F01758E0474F6
:10664B0080D5E0FD438902E58930E4FB759702753F
:10665B00840075D10775840075BB0175BA0075BCD4
:10666B00F075C70075C60075C5FF75C4FF75E800EA
:10667B0075840275BB0475BA0075BCF175C60075DF
:10668B00C4FF75E88075840075D48475840175D456
:10669B0084758400C2F8759A47759D1A75F8017553
:1066AB00870075840075B90075A900759100759800
:1066BB005075840175989075840075C04075C30042
:1066CB0075CFC9758400758E107589217588057510
:1066DB008400758A00758BE0758CF4758DE04388AA
:1066EB004075840075C90075CA0075CB0075CC0068
:1066FB0075CD0075840175C91875CA8075CBFB758E
:10670B00CDFB75CC80D2CA75840275C91875CAA623
:10671B0075CBAF75CDAF75CCA6D2CA75840075EFAE
:10672B000275A8AC75B83D75E6B075E71D75F6003A
:10673B0075F741789B760A769C780A789D76067574
:07674B00A8959000007F00FB
:106752007E20E4F0A3DFFCDEFA789B760A789C7652
:0E6762000A789D7606D29375E8FF1275212203
:10796F0075840FD2FD2275840FC2FD22E490FC00B6
:10797F00732275840FD2EA2275840FC2EA227584AE
:10798F000FA2EC2275840FD2FC2275840FC2FC2249
:10799F0075840FC2FF2275840FD2FF2275840FA248
:1079AF00FA2275840FA2F92275840FA2DD22A2920A
:1079BF002275840FA2DA2275840FA2DB2275840F41
:1079CF00A2D82275840FA2D9220000000000000067
:1079DF000000000000000000000000000000000098
:1079EF00000000000022C000C001790878B4D8FE62
:1079FF00D9FAD001D00022C000C0E078977605E612
:107A0F0070FDD0E0D00022C000C0E07897760FE67E
:107A1F0070FDD0E0D00022C000C0E078977664E619
:107A2F0070FDD0E0D00022EF75F064842430900018
:107A3F0054F0E5F0A375F00A842430F0A3E5F024A8
:107A4F0030F022EF75F064842430900054F0E5F0AC
:097A5F00A375F00A842430F0A3A1
:107A6800E5F02430F0900054E0B4300B7420F0A31B
:107A7800E0B430037420F02275F06484F6E5F00871
:107A880075F00A84F608A6F00822850607222285E2
:037A9800050622BE
:101A1A00C0D0C000C001C083C082C0E0C0F0C0070F
:101A2A00A291304F01B37825E233F208E233F2088B
:101A3A00E233F208E233F208E233F208E233F20860
:101A4A00E233F208E233F208E233F208E233F20850
:101A5A00E233F208E233F208E233F208E233F20840
:101A6A00E233F208E233F208E233F208E233F20830
:101A7A00E233F208E233F208E233F208E233F20820
:101A8A00E233F208E233F208E233F208E233F20810
:101A9A00E233F208E233F208E233F208E233F20800
:101AAA00E233F208E233F208E233F208E233F208F0
:011ABA00E249
:101ABB0033F208E233F208E233F208E233F208E2DF
:101ACB0033F208E233F2305B32784CE218203C03FD
:101ADB0030E728E21820E723E21830E71EE218204F
:101AEB00E719E21830E714E21830E70FE21820E7A5
:101AFB000AE21820E705E21830E703021C5E754086
:101B0B0000E2183392475003754038752200E218F3
:101B1B00339214500363401CE21833921350036347
:101B2B00400EE2183392125003634046E218339290
:101B3B00115003634023E218339210852241500366
:101B4B00634051752200E2183392145003634068CE
:101B5B00E2183392135003634075E218339212501C
:101B6B000363407AE218339211500363403DE2184D
:101B7B00339210852242500363401F752200E218F6
:101B8B00339217500363404FE2183392165003639E
:101B9B004026E2183392155003634052E2183392F9
:071BAB00145003634029E21E
:101BB200183392135003634015E218339212500304
:101BC20063400BE2183392115003634045E218332D
:101BD20092108522435003634062E21833921450FC
:101BE20003634031E2183392135003634019E21841
:101BF200339212500363400DE21833921150036383
:101C02004007E21833921085224450036340437523
:101C12002200E218339216E218339215E218339238
:101C220014E218339213E218339212E2183392112B
:101C3200E218339210852245E5456540701EA247A1
:101C4200924890004DE541F090004EE542F0900040
:101C52004FE543F0900050E544F0D24A121C72D096
:101C620007D0F0D0E0D082D083D001D000D0D022F3
:101C7200C0D0C000C0E0303F4EE552B40833A242AB
:101C8200B392B3787BE66036167880E6A2E73044FA
:101C920001B3924292B2A2E7787CE633F6787DE60F
:0C1CA20033F6787EE633F6787FE633F602
:101CAE007880E633F6D55203755208D0E0D000D0D6
:101CBE00D022C257D0E0D000D0D022D0E0D000D079
:101CCE00D022C0D0C000C001C083C082C0E0C0F02E
:101CDE00A291204E01B3780DE213F208E213F2083E
:101CEE00E213F208E213F208E213F208E213F2082A
:101CFE00E213F208E213F208E213F208E213F2081A
:101D0E00E213F208E213F208E213F208E213F20809
:101D1E00E213F208E213F208E213F208E213F208F9
:101D2E00E213F208E213F208E213F208E213F208E9
:101D3E00E213F2901E85780DE2089313920FE208DB
:101D4E009313920EE2089313920DE2089313920CE2
:081D5E00E2089313920BE20866
:101D66009313920AE20893139209E20893139208D6
:101D7600852146E2089313920FE2089313920EE22E
:101D8600089313920DE2089313920CE208931392B0
:101D96000BE2089313920AE20893139209E208935E
:101DA600139208852147E2089313920FE2089313D2
:101DB600920EE2089313920DE2089313920CE20836
:101DC6009313920BE2089313920AE2089313920973
:101DD600C208852148305B3DE5469021D5854721DF
:101DE600300E02058393602D14F875F003A490203D
:101DF600862582F582E5F03583F583E493F9A3E43D
:101E060093901F85654893C965479329B40100508F
:101E1600048834D241121E2DD0F0D0E0D082D08377
:101E2600D001D000D0D022303D27C392B27881169F
:101E3600E6701E76087884E6A2E1304501B392B3D7
:101E4600A2E17882E613F67883E613F67884E61341
:101E5600F622EF90208575F003A42582F582E583AE
:101E660035F0F583C23D7400937882F67401937859
:101E760083F67402937884F6C23FC23ED23D2200B6
:101E8600000000000000000000000000000000004C
:101E9600000000000000000000000000000001003B
:101EA600000000000000000000000000000001002B
:101EB6000000000000000100000001000101010017
:101EC600000000000000000000000000000001000B
:101ED60000000000000001000000010001010100F7
:101EE60000000000000001000000010001010100E7
:101EF60000000100010101000101010101010100D1
:101F060000000000000000000000000000000100CA
:101F160000000000000001000000010001010100B6
:101F260000000000000001000000010001010100A6
:101F36000000010001010100010101010101010090
:101F46000000000000000100000001000101010086
:101F56000000010001010100010101010101010070
:101F66000000010001010100010101010101010060
:101F7600010101010101010101010101010101004C
:101F8600010102010202030102020302030304012A
:101F9600020203020303040203030303030405010D
:101FA60002020302030304020303040304040502FA
:101FB60003030403040405030404040405050601DD
:101FC60002020302030304020303030304040502DB
:101FD60003030403030405030404050405050602BC
:101FE60003030403040405030404050405050603AA
:101FF600040405040505060405050605060607018D
:102006000202030203030402030304030404050299
:10201600030304030404050304040504050506027A
:102026000303040304040503040405040505060369
:10203600040405040505060405050605060607024B
:102046000303040304040503040405040505060349
:10205600040405040505060405050605060607032A
:102066000404050405050604050506050606070419
:10207600050506050606070506060706070708FD01
:10208600D00C73700E3CF01AAF101E7F9022EC70CD
:1020960026D6F02ACBB02CA3F032BEB03417D03CF3
:1020A600B6D0461FB04E77F050F950526AB056DEA1
:1020B6009058BA306ACF3072D270745CD076E8F03D
:1020C600786BD098E5709AF8309CBB50A40F70AA34
:1020D6007A70B26730B45DB0B8FCB0C26F50C65506
:1020E600D0CA3D90D489B0DA94F0DCD790E463B0DE
:1020F600EA0BF0F43170F8DD310AB571148FF1187E
:10210600D1D126EB512AF6112C8B71463F5148B19D
:10211600F14AACB14CC4F152D9B1546D915A2EF179
:1021260062BD116687916A9AD16CF29172D5517827
:1021360019F18C71B192D8D19A32D1AA47D1B25A3B
:1021460091B452F1C67531CC1D71D2A951DCD0B112
:10215600E85E11EA2B11F2EED212F392147D3216DA
:10216600973226D8B232C5F234F7124AEA524C9F59
:102176005254A5D2582B725A7552644FD268C17206
:102186006ADC326C78D2865F128C83729C4EB2A661
:102196006972AC1C72B433D2CC18F2EABB330CCEE3
:1021A60033141EB32803F32EE51332F85334987311
:0D21B6005848F36472736845738617B3943C
:1021C3007313A63C93B221D3B41B53B829B3C641AE
:1021D300F3D8000000000000000000000000000031
:1021E3000000000000000000006A00000000000082
:1021F300620D0000000000000000006F00480000B6
:1022030000000000000000000000000000006C223D
:1022130000000000000000000000000000000000BB
:102223005B00000000000000000000004100001EF1
:102233004759000000260000001D00001000003573
:102243000000003D006B0043000000000000004B55
:10225300000500000000000000380023000000001B
:102263000000000000000000004C0000000000001F
:102273000000000000000000000000000000320029
:10228300000400000000000000000000126000379E
:102293000A00000000000000000000000008000029
:1022A300611346000000000000254D34000057294B
:1022B30011000000000000640000000000000000A6
:1022C300000000003A4A00002E4F190000001F00D2
:1022D3000000000000630000000000000027000071
:1022E300001B000000000000000B5F3C006E5D441B
:1022F3000000006D0000000000000000005300001B
:10230300360000283F5E00000000000000000300CC
:10231300003000700000006900406700000000000A
:1023230000550000420000210000000000001500DD
:1023330000000000000000000000005C0017000027
:102343000020000068020054000E58001C0000002A
:1023530000000000005A000000000000002F0000F1
:10236300002B00000000240000006600390000007C
:102373000051000000090052000000450000000069
:10238300000000310000002A0C000000001A0000C9
:10239300000000560000334E000000000000000063
:1023A3000000002C1400003B07003E00000000006A
:1023B300000000000000001800001600502D060069
:1023C30049000000000000000000650F000000014C
:1023D30000000000000000000600000006000600E8
:1023E30005020600060006000404060005040208B0
:1023F30006000000060006000600060004080600AA
:102403000600060005080600060002100600060086
:102413000301000006000600020206000600044055
:10242300060006000410060006000600060006006B
:10243300060006000510060006000600060006005A
:10244300060001010600060006000600030206005E
:10245300060000000600060005010600040202044F
:102463000600060006000600060006000600060039
:102473000480060002010420060006000600060090
:102483000600060006000600060006000600060019
:10249300060006000600040106000600060006000A
:1024A30006000310060006000600060006000600EC
:1024B30006000600060006000600060003080600E4
:1024C30006000600060003040600060006000600D8
:0224D300060001
:10596400758400C2CA85CC3885CD3775CC0075CD19
:1059740000D2CA10CF02D25A32305A0BC25AE5377B
:10598400C394364002800122788C798A7B06E7F63C
:105994001819DBFAA63718A638AA38AB37AE02AF07
:1059A40003EEC4035407FEEFC403FF54F84EFEEFA6
:1059B4005407FF78037987C3E79AFC09E79BFD093D
:1059C40050066304FF6305FFC3EC9EED9F5074D83B
:1059D400E6789479927C06E7F61819DCFAA603189F
:1059E400A602798FAE02AF03EEC423541FFEEFC4A8
:1059F40023FF54E04EFEEF541FFF7803C3E79AFCE5
:105A040009E79BFD0950066304FF6305FFC3EC9E91
:105A1400ED9F502FD8E6788D7A007B007C007904C6
:105A2400EA26FA08EB36FB08EC3400FCD9F2EC1356
:0D5A3400FCEB13FBEA13FAEC13EB13F53651
:105A4100EA13F535D23A22303A31C23A125A7D5030
:105A51002A853C3D853B3C853A3B85393A8507396A
:105A6100303913E53F6F600EE507B53A0EB53B0BD4
:105A7100B53C08B53D0585073ED23B22905B98E5D4
:105A81003693FF905AC423232582F582E58334009F
:105A9100F583125AA3400A0F125AA340040F125A57
:105AA100A322E493F9A3E493FAA3E493FBA3E4937D
:105AB100FCA3C3E5359AE536995007C3EC9535EB60
:105AC100953622EA25DD89DD89D324D324CBD2CBB7
:105AD100D2C4DBC4DBBE39BE39B7CAB7CAB18EB1D5
:105AE1008EAB87AB87A59CA59CA000A0009A969A37
:105AF1009695D895D891E591E58D858D8588AF8866
:105B0100AF840C840C7F9A7F9A7B497B49771B7702
:105B11001B730F730F6F276F276B576B5767AB673C
:105B2100AB642C642C60C660C65D795D795AFE5AFF
:105B3100FE5970597057E257E25661566154E75465
:105B4100E7537453745207520750A050A04F404F6F
:105B5100404DE64DE64C934C934B414B4149F54941
:105B6100F548B548B547764776463E463E45084531
:105B710008432A432A40E440E43F533F533E3E3E1C
:105B81003E3C943C943A863A8639183918380500D7
:105B91000000000000000032323232323232323242
:105BA10032323232323232323232323232323232D4
:105BB10032323232323232323232323232323232C4
:105BC10032323232323232323232323232323232B4
:105BD100313130302F2E2D2D2D2C2C2B2A292928F7
:105BE10027262525242323222120201F1E1E1D1C9C
:105BF1001C1B1A1A1A1A1919191818181717171716
:105C0100161616161515151514141414131313134B
:105C1100121212121111111110101010100F0F0F7A
:105C21000F0F0E0E0E0E0D0D0D0D0C0C0C0C0B0BA3
:105C31000B0B0B0B0A0A0A0A0A09090909090908C7
:105C410008080808080707070707070606060606E3
:105C510006060505050505050404040404040403FA
:105C61000303030303030202020202020201010110
:105C71000101010101010101010101000000000018
:105C81000000000000000000000000000000000013
:075C9100000000000000000C
:1071EC00C007C0007F01127EC27F4C127E937F5479
:1071FC00127E937F52127E937F20127E932049043D
:10720C007F3080027F31127E937F20127E9390011B
:10721C0091E0784B127A88784B8607430730127EC0
:10722C0093088607430730127E93750720127E93CE
:10723C00900192E0784B127A80784B8607430730A6
:10724C00127E93088607430730127E930886074305
:10725C000730127E93750720127E93900193E0788D
:10726C004B127A88784B8607430730127E93088638
:10727C0007430730127E93750720127E93D000D0FF
:10728C000722C007C0007F11127EC27F4C127E9372
:10729C00750720127E93204D047F3080027F3112BF
:1072AC007E937F20127E9390015BE0784B127A885C
:1072BC00784B8607430730127E93088607430730C6
:1072CC00127E93750720127E9390015CE0784B122E
:1072DC007A80784B8607430730127E9308860743E3
:1072EC000730127E93088607430730127E9375078A
:1072FC0020127E9390015DE0784B127A88784B8651
:10730C0007430730127E93088607430730127E939B
:10731C00750720127E9390015EE0784B127A887884
:10732C004B8607430730127E9308860743073012BB
:07733C007E93D000D0072270
:106F2E00003800512372461765340E5F2D7C4819C8
:106F3E006B3A1C4D3F6E5A0B792812433160540543
:106F4E007726001F3D227A654758756A48570F10FD
:106F5E00322D6877554A120D2F301D02203F67786B
:106F6E005A45006245270B694E2C157750321E7C10
:106F7E005B39294B6C0E224067053C5E791B3755F9
:106F8E00721052301775593B1C7E472502604C2EED
:106F9E00096B7B193E5C701235576E0C2B496507D9
:106FAE002042264463012D4F680A33517614385A15
:106FBE007D1F0F6D4A28046641231A785F3D1173B9
:106FCE005436741631537F1D3A58610324466A08AD
:106FDE002F4D5D3F187A56341371482A0D6F432199
:106FEE0006644F2D0A68442601635A381F7D5133BB
:106FFE001476660423416D0F284A73113654781A9D
:10700E003D5F1D7F583A16745331086A4D2F036148
:10701E004624345671133F5D7A18214364062A487C
:10702E006F0D690B2C4E620027457C1E395B771560
:10703E003250402205674B290E6C553710725E3C5C
:10704E001B793B597E1C305275172E4C6B09254708
:10705E00600212705735197B5C3E076542200C6E3C
:10706E00492B004307440D4E0A49195A1E5D145709
:10707E001350317236753C7F3B78286B2F6C25662A
:02708E0022617D
:10867F00788076ACA24DE433FFC4333354C0FE9000
:10868F00015DE0FD541F25E04EFE90015BE0FC54C0
:10869F0010C4540F4E787FF6EC540FC454F0FE9074
:1086AF00015CE0FC54F0C4540F4E787EF6EC540F8E
:1086BF00C454F0FE90015EE0FC541EC3134E787D4F
:1086CF00F6EF3395E0FE742E2FF582746F3EF5832F
:1086DF00E493FFED906F3093FEEF6EFF90015BE040
:1086EF00906F50936FFF90015CE0906F70936FFFEE
:1086FF00EC907070936F787CF690015EE030E00440
:0B870F00E64480F6D257787B762822E3
:10923700758401309914C29920500F900159E0703C
:1092470009D250D29C789576042230983790015AEB
:10925700E06401702DE54975F0058420551124EF70
:10926700F582E43400F583E599F0C298D2552224BB
:1092770004F582E43401F583E599F0C298C255D22A
:059287005622C29822EE
:1081F2007584012098030282B8205213209A0DE55B
:10820200997009D252D253754A0AF549C2982290FE
:10821200015AE0FF6401702CE54975F00584205590
:108222001024EFF582E43400F583E599F0D255800D
:10823200102404F582E43401F583E599F0C255D2A5
:1082420056C29822EFB4021AAB530555E555AA540B
:108252007002055414F9E59912861F90015A7403AD
:10826200802090015AE0FFB4031CAB530555E5553D
:10827200AA547002055414F9E59912861F90015A06
:108282007404F0C29822EFB4042990018CE0FF0438
:10829200F074632FF582E43401F583E599F0C29816
:1082A20090018CE0B4281C90018E7401F0E49001DE
:1082B2005AF022C2982230990AC299900159E0706C
:0482C20002C255227D
:1099E6002051221279A543E740754A0AE4F54990C9
:1099F6000159F090015AF0C250D251758401759800
:069A060090C29CF59922BC
:10900D0090018DE0705C9001ABE0FF7025D3900175
:10901D0060E0948690015FE094674008E4F0A374EB
:10902D0002F0800E900160E02428F090015FE034A2
:10903D0000F0900160E02FFF90015FE03400FE1220
:10904D0074D89001ABE02463F582E43401F583EF2D
:10905D00F09001ABE004F0E0B42807E4F090018D4E
:03906D0004F022EA
:108B890090018EE0607A900161E0FEA3E0FFC3945A
:108B990002EE94005006E490018EF0229001ABE0C1
:108BA9007C002FFFEC3EFE1274D89001ABE02463E9
:108BB900F582E43401F583E0FD6F60179001ABE0C5
:108BC900FF900162E02FFF900161E03400FE127412
:108BD90097D2549001ABE004F0E0B42823E490016B
:108BE9008EF09001ABF0900161E07004A3E06402A3
:108BF900700E30540BC2541288451290D012912C29
:018C09002248
:108ED8003050647584019001A0E0B40D00505590A5
:108EE8008EEEF8282873028F15028F18028F1B0246
:108EF8008F1E028F21028F24028F27028F2A028F52
:108F08002D028F30028F33028F36028F3902993348
:108F1800029B480294A20296A5029A0C02005E02E5
:108F280098CF0297FC0296E10294E5029AE702992B
:088F38008E029ACC129B01226B
:109933007895E67028759898754A0AF54990005B02
:10994300E0B401079001A07404F022E490015AF0FE
:0E995300900159F09001A0E004F012799F22DB
:109B480090015A7401F0E4900159F0C2559001A0B7
:049B5800E004F02213
:1094A20090005BE01475F005A4B54919E4B5F01518
:1094B2007598981279A5E4900159F090015AF090AC
:1094C20001A07404F0E54975F00584AFF0BF011204
:1094D200C256E4900159F090015A04F09001A0E0C4
:0394E20004F02271
:1096A500E54975F00584AFF0BF043020561EE54945
:1096B50075F00584FF24EFF582E43400F583E4F0CA
:1096C50074042FF582E43401F583E4F0E490015944
:0C96D500F090015AF09001A0E014F02287
:109A0C0090005BE075F005A424FDB549159000525B
:109A1C00E0F599E4900159F090015AF09001A0E022
:039A2C0004F02221
:0D005E00900053E0F5999001A0E004F0221D
:1098CF0090005BE0FD75F005A4FFE549B50723E4C3
:1098DF00B5F01FEDB414079001A07409F0221279AE
:1098EF009FE4900159F0C25590015AF09001A0E009
:0398FF0004F02250
:1097FC00E549B464121279A5E4900159F090015A2C
:10980C00F09001A07409F0E54975F00584AFF0BF44
:10981C000112C256E4900159F090015A04F09001E3
:05982C00A0E004F022A1
:1096E100E54975F00584AFF0BF043020561EE54909
:1096F10075F00584FF24EFF582E43400F583E4F08E
:1097010074042FF582E43401F583E4F0E490015907
:0C971100F090015AF09001A0E014F0224A
:1094E500E5496465703C90018DE0B4012F75530129
:1094F50075540175555FE4900159F090015AF07566
:109505008401AB530555E555AA547002055414F969
:109515001285D9F5999001A0E004F0229001A0747C
:039525000CF02225
:109AE700758401AB53AA54A9551285D9F599E49009
:0A9AF700018BF09001A0E004F022C2
:10998E0075840190018BE0FF04F074632FF582E47F
:10999E003401F583E0F59990018BE0D39428400BC8
:0C99AE00E490018DF09001A0E004F02294
:109ACC00E549B46915C250C251E49000EDF0900123
:0B9ADC0059F090015AF09001A0F02218
:109B0100C250C251E4F5499000EDF0900159F09036
:089B1100015AF09001A0F022BE
:1091E1003052527584019001A1E0B40A00504390BD
:1091F10091F7F828287302921502921802921B0225
:10920100921E02922102922402922702922A029233
:109211002D0292300297C602971D029756029A8F2D
:10922100029BB80299BA0295AD02978E029A2F025B
:069231009BA7129BC8225E
:1097C600E549703175989890005BE0B40113127901
:1097D600A5E490015AF0900159F09001A17403F0AC
:1097E6002212799FC255E490015AF0900159F090E7
:0697F60001A1E004F022D5
:10971D0090005BE01475F005A4B54911E4B5F00DAA
:10972D007598981279A59001A17403F022E54975F9
:10973D00F00584AFF0BF0110C256C25590015A74A6
:09974D0001F09001A1E004F022FA
:10975600E54975F00584AFF0BF042C20561EE54997
:1097660075F00584FF24EFF582E43400F583E4F018
:1097760074042FF582E43401F583E4F0E490015A91
:08978600F09001A1E014F022B3
:109A8F0090005BE075F005A424FDB54911758401C4
:0F9A9F00900052E0F599C2559001A1E004F02229
:109BB800758401900053E0F5999001A1E004F0222A
:1099BA0090005BE0FFB414079001A17406F022EF57
:1099CA0075F005A4B54914E4B5F01012799F900119
:0C99DA00A1E004F0C255E490015AF02214
:1095AD00E54975F00584AFF0BF0111C256C2559063
:1095BD00015A7401F09001A1E004F022E549B46470
:1095CD001F12799F90018EE0700B90015AF090015F
:1095DD00A17408F022E490015AF09001A17409F0F1
:0195ED00225B
:10978E00E54975F00584AFF0BF042C20561EE5495F
:10979E0075F00584FF24EFF582E43400F583E4F0E0
:1097AE0074042FF582E43401F583E4F0E490015A59
:0897BE00F09001A1E014F0227B
:109A2F00E549B4651A755301755401755561E49094
:109A3F00018CF09001A17409F090015A7402F02288
:109BA700E549B4690BC252E490015AF09001A1F063
:019BB700228B
:109BC800C252E490015AF0900159F09001A1F0229C
:1082C6007898E6600116900000E0600214F09000D5
:1082D60001E0600214F0900002E0600214F09000E9
:1082E6000BE0600214F090000AE0600214F0789A45
:1082F60016E66003028399789A760A7899E6600111
:1083060016900004E0600214F0900005E06002148C
:10831600F0900006E0600214F0900008E06002149D
:10832600F0900009E0600214F0789EE66001169075
:108336000003E0600214F09001E7E0600214F078B8
:108346009B16E6704E789B760A90000CE06002144D
:10835600F078A0E61846600708E616187001169031
:1083660001A3E0600214F09001A4E0600214F09012
:1083760001A7E0600214F0789C16E67016789C76E9
:108386000A789D16E6700C789D76069001A6E06048
:048396000214F022BB
:106AC500535155452020434F53202053454E5345A0
:106AD500004F4E2020202020202020202020202074
:106AE50020004F4646202020202020202020202046
:106AF5002020002020205245504541544552203148
:106B05002020200020202052455045415445522048
:106B15003220202000202020524550454154455226
:106B25002033202020002020205245504541544547
:106B35005220342020200020202052455045415429
:106B45004552203520202000202020524550454127
:106B55005445522036202020002020205245504503
:106B650041544552203720202000202020524550F6
:106B750045415445522038202020002020205245F0
:106B850050454154455220392020200020202052D4
:106B950045504541544552203130202000202020C9
:106BA5005245504541544552203131202000202086
:106BB5002052455045415445522031322020002075
:106BC5002020524550454154455220313320200064
:106BD5002020205245504541544552203134202033
:106BE5000020202052455045415445522031352042
:106BF5002000202020524550454154455220313631
:106C05002020002020205245504541544552203136
:106C15003720200020202052455045415445522020
:106C250031382020002020205245504541544552FE
:106C3500203139202000202020524550454154451F
:076C45005220323020200034
:10002E00750C01E50CC394155018AF0C74182FF510
:10003E0082E43401F583E0FFEF60037F0122050CBB
:04004E0080E17F00CE
:01005200228B
:10918800205755128468EF6401704D90009AE0FFF3
:10919800EF24FF924D900158E0FF74422FF582E4CE
:1091A8003401F583E0FF90015BEFF0900158E0FF98
:1091B800742D2FF582E43401F583E0FF90015CEF14
:1091C800F0900158E0FF90015DEFF0126405900106
:0991D8005EEFF012867FD23F2207
:108468009000E8E4F0A3E4F09000EBE4F0A3E4F07B
:108478009000E7E4F09000E7E0FFEFC394154003B5
:1084880002850C900158E0FFEFD394144006900148
:10849800587401F0900158E0FF74182FF582E43405
:1084A80001F583E0FF9000EAEFF09000EAE0FFEFCB
:1084B800B40115900158E0FF74182FF582E43401D7
:1084C800F5837402F07F01229000EAE0FFEFB40226
:1084D800249000E8E0FEA3E0FFEF4E70189000E85B
:1084E800E4F0A37401F0900158E0FF7E009000EBE7
:1084F800EEF0A3EFF0900158E004F09000E7E004FC
:10850800F002847D9000E8E0FEA3E0FFEF4E7004E7
:108518007F0022229000ECE0FF900158EFF07F01ED
:018528002230
:10839A009000E8E4F0A3E4F09000EBE4F0A3E4F04A
:1083AA009000E7E4F09000E7E0FFEFC39415400384
:1083BA0002844B900158E0FFEFD3941440069001D9
:1083CA00587401F0900158E0FF74182FF582E434D4
:1083DA0001F583E0FF9000EAEFF09000EAE0FFEF9A
:1083EA00605090005BE0FF900158E0FEEE6F604243
:1083FA009000EAE0FFEFB40115900158E0FF74180D
:10840A002FF582E43401F5837402F07F0122900093
:10841A00E8E0FEA3E0FFEF4E7018900158E0FF7EFF
:10842A00009000EBEEF0A3EFF09000E8E4F0A37404
:10843A0001F0900158E004F09000E7E004F00283B4
:10844A00AF9000E8E0FEA3E0FFEF4E70047F002249
:0E845A00229000ECE0FF900158EFF07F01222D
:1064050090005BE0FFEFD3941440037F20229001BE
:10641500EDE4F09001ECE4F090005BE0FF9001EA20
:10642500EFF0900095E0FFEFD3940650030264F976
:106435009001EBE4F09001EBE0FFEFC3941540030E
:106445000264F29001EAE0FFEFB415069001EA74E8
:1064550001F09001EAE0FF74EE2FF582E43400F5D7
:1064650083E0FFEF64FF70769001EAE0FF74BE2FD2
:10647500F582E43400F583E0FF90005BE0FE74BE36
:106485002EF582E43400F583E0FEEEC39F404F9085
:10649500005BE0FF9001EAE0FEEEB507069001EA39
:1064A500E0FF229001EAE0FF74BE2FF582E434009C
:1064B500F583E0FF9001ECE0FEEFD39E40209001D4
:1064C500EAE0FF9001EDEFF09001EAE0FF74BE2FE6
:1064D500F582E43400F583E0FF9001ECEFF09001E4
:1064E500EBE004F09001EAE004F002643A9001ED7B
:1064F500E0FF22229001EBE4F09001EBE0FFEFC317
:10650500941540030265B59001EAE0FFEF7006902F
:1065150001EA7414F09001EAE0FF74EE2FF582E4CD
:106525003400F583E0FFEF64FF70769001EAE0FF49
:1065350074BE2FF582E43400F583E0FF90005BE044
:10654500FE74BE2EF582E43400F583E0FEEEC39FB3
:10655500404F90005BE0FF9001EAE0FEEEB50706D4
:106565009001EAE0FF229001EAE0FF74BE2FF58278
:10657500E43400F583E0FF9001ECE0FEEFD39E40AC
:10658500209001EAE0FF9001EDEFF09001EAE0FFD5
:1065950074BE2FF582E43400F583E0FF9001ECEF43
:1065A500F09001EBE004F09001EAE014F00264FEE3
:0565B5009001EDE0FF84
:0165BA0022BE
:1069250090005BE0FFEFD3941440037F2022900199
:10693500F1E4F09001F0E4F0900095E0FFEFD394DE
:10694500065003026A0A90005BE0FFEF04FF900126
:10695500EEEFF09001EFE4F09001EFE0FFEFC3946C
:10696500154003026A039001EEE0FFEFD394144053
:10697500069001EE7401F09001EEE0FF74EE2FF544
:1069850082E43400F583E0FFEF64FF70629001EE6E
:10699500E0FF74BE2FF582E43400F583E0FF90003C
:1069A5005BE0FE74BE2EF582E43400F583E0FEEE76
:1069B500C39F403B9001EEE0FF74BE2FF582E434A7
:1069C50000F583E0FF9001F0E0FEEFD39E402090BC
:1069D50001EEE0FF9001F1EFF09001EEE0FF74BEF3
:1069E5002FF582E43400F583E0FF9001F0EFF0909D
:1069F50001EFE004F09001EEE004F002695D900122
:106A0500F1E0FF222290005BE0FFEF14FF9001EE22
:106A1500EFF09001EFE4F09001EFE0FFEFC3941584
:106A25004003026ABF9001EEE0FFEF70069001EEB1
:106A35007414F09001EEE0FF74EE2FF582E434005B
:106A4500F583E0FFEF64FF70629001EEE0FF74BE36
:106A55002FF582E43400F583E0FF90005BE0FE74DF
:106A6500BE2EF582E43400F583E0FEEEC39F403B85
:106A75009001EEE0FF74BE2FF582E43400F583E06B
:106A8500FF9001F0E0FEEFD39E40209001EEE0FF85
:106A95009001F1EFF09001EEE0FF74BE2FF582E476
:106AA5003400F583E0FF9001F0EFF09001EFE00492
:0F6AB500F09001EEE014F0026A1C9001F1E0FF96
:016AC40022AF
:1067700090005BE0FFEFD3941440037F2022900051
:1067800052E0FFEFB4FF0C900053E0FFEFB4FF03C3
:106790007F00229001F5E4F09001F4E4F090009580
:1067A000E0FFEFD39406500302686A90005BE0FFBD
:1067B000EF04FF9001F2EFF09001F3E4F09001F3A9
:1067C000E0FFEFC3941540030268639001F2E0FF1D
:1067D000EFD3941440069001F27401F09001F2E0BE
:1067E000FF74EE2FF582E43400F583E0FFEF64FFE1
:1067F00070629001F2E0FF74BE2FF582E43400F580
:1068000083E0FF90005BE0FE74BE2EF582E434006E
:10681000F583E0FEEEC39F403B9001F2E0FF74BEC3
:106820002FF582E43400F583E0FF9001F4E0FEEF01
:10683000D39E40209001F2E0FF9001F5EFF090012F
:10684000F2E0FF74BE2FF582E43400F583E0FF90A0
:1068500001F4EFF09001F3E004F09001F2E004F0B5
:106860000267BD9001F5E0FF222290005BE0FFEFA0
:1068700014FF9001F2EFF09001F3E4F09001F3E0E7
:10688000FFEFC39415400302691F9001F2E0FFEF90
:1068900070069001F27414F09001F2E0FF74EE2F94
:1068A000F582E43400F583E0FFEF64FF706290014D
:1068B000F2E0FF74BE2FF582E43400F583E0FF9030
:1068C000005BE0FE74BE2EF582E43400F583E0FE4A
:1068D000EEC39F403B9001F2E0FF74BE2FF582E4CF
:1068E0003400F583E0FF9001F4E0FEEFD39E4020FA
:1068F0009001F2E0FF9001F5EFF09001F2E0FF74FB
:10690000BE2FF582E43400F583E0FF9001F4EFF050
:106910009001F3E004F09001F2E014F002687C9042
:0469200001F5E0FF9E
:016924002250
:109B5C0090005BE0FFEFD3941440037F2022900031
:049B6C005BE0FF2299
:10784100900157E0FFEFD394144006900157740163
:10785100F09000E7E4F0900157E0FF742D2FF582DE
:10786100E43401F583E0FF900157E0FE74032EF547
:1078710082E43401F583E0FEEEB50726900157E07E
:10788100FF74422FF582E43401F583E0FF90015744
:10789100E0FE74EE2EF582E43400F583E0FEEE6F37
:1078A10060069000E77401F0900157E0FF74EE2F3D
:1078B100F582E43400F583E0FF90005BE0FEEF6EBB
:1078C100600E90005BE0FF900157E0FEEE6F703AB2
:1078D1009000E7E0FFEF6043900157E0FFEFD394A2
:1078E100155014900157E0FF74182FF582E434010C
:1078F100F5837401F08024900157E0FF74182FF58F
:1079010082E43401F583E4F08011900157E0FF74C3
:10791100182FF582E43401F583E4F09000E7E0FFED
:10792100EF6044900157E0FF74032FF582E43401C6
:10793100F583E0FF900157E0FE742D2EF582E434CB
:1079410001F583EFF0900157E0FF74EE2FF582E42B
:107951003400F583E0FF900157E0FE74422EF5827A
:0E796100E43401F583EFF0900157E004F022CA
:10734300900198E0FFEF60030273F1900006E0FF05
:10735300EF70037F012212956BEFB401051279815F
:107363008003127987204A037F002212956BEF6412
:10737300017078304A72C24A1271EC90004EE0FFFD
:10738300900194EFF090004FE0FF900195EFF090A3
:10739300004DE0FF900196EFF0900196E0FFEFB40F
:1073A3001F14900192E0FF900195E0FEEEB50706F1
:1073B3001279877F0122900191E0FF900194E0FE12
:1073C300EEB5070E900192E0FF900195E0FEEE6F9F
:1073D30060099001987401F07F002290008CE0FF17
:1073E300900006EFF07F00227F00227F00229001B1
:1073F30098E0FFEF6401600302748F900006E0FFE2
:10740300EF70037F012212956BEFB40105127981AE
:107413008003127987204A037F0022C24A1271EC4B
:1074230090004EE0FF900194EFF090004FE0FF904A
:107433000195EFF090004DE0FF900196EFF0900181
:1074430096E0FFEFB41F14900192E0FF900195E0E6
:10745300FEEEB507061279877F0122900191E0FFC6
:10746300900194E0FEEEB50720900192E0FF9001B9
:1074730095E0FEEEB5071290008CE0FF900006EF5A
:10748300F0900198E4F07F00227F0022900198E4BD
:04749300F07F002264
:10956B00900083E0FFEF600D1279AB40047F018028
:10957B00027F002222900084E0FFEF6013900085B1
:10958B00E0FFE532D39F40047F0122227F0022229D
:10959B00900085E0FFE532C39F50047F0122227FBC
:0295AB0000229C
:1070900090019DE0FFEF6003027142900008E0FF65
:1070A000EF70037F012212956BEFB4010512798115
:1070B000800312798790019CE0FFEFB40106203B2A
:1070C000037F002290019CE0FFEFB4020620410301
:1070D0007F002212956BEF6401706490019CE0FFC9
:1070E000EF64017021303B1EC23BE53F653E600905
:1070F00090019D7401F07F0022900091E0FF9000CC
:1071000008EFF07F002290019CE0FFEF6402702FF7
:1071100030412CC24190019FE534F090019FE0FF87
:1071200090019EE0FEEE6F600990019D7401F07F7A
:107130000022900091E0FF900008EFF07F00227F96
:10714000002290019DE0FFEF640160030271EB906B
:107150000008E0FFEF70037F012212956BEFB4018E
:1071600005127981800312798790019CE0FFEFB4CA
:107170000106203B037F002290019CE0FFEFB40258
:10718000062041037F002212956BEF6401705A9034
:10719000019CE0FFEFB4011C303B19C23BE53FB559
:1071A0003E1290019DE4F0900091E0FF900008EF06
:1071B000F07F002290019CE0FFEF6402702B3041D1
:1071C00028C24190019FE534F090019FE0FF9001BB
:1071D0009EE0FEEEB5071290019DE4F0900091E074
:0C71E000FF900008EFF07F00227F0022EB
:108F40007BFF7A6A79C51298311279AB400B7BFFAF
:108F50007A6A79D612986680097BFF7A6A79E71275
:108F600098667F17127EC2AF32127A52900054E098
:108F7000FF127E93900055E0FF127E93900056E022
:108F8000FF127E937F1C127EC2AF31127A52900084
:108F900054E0FF127E93900055E0FF127E93900004
:078FA00056E0FF127E932250
:10996100900088E0FFEF6013900089E0FFE531D3BC
:109971009F40047F0122227F002222900089E0FF84
:0D998100E531C39F50047F0122227F0022A8
:109BD800900083E0FFEF6004128C0A22126DCA2203
:108C0A009001A5E0FFEF70161279AB4072900086D2
:108C1A00E0FF90000AEFF09001A5E004F022900135
:108C2A00A5E0FFEF640170281279AB401C90000A9E
:108C3A00E0FFEF704AD25B900090E0FF900007EFF0
:108C4A00F09001A5E004F022229001A5E4F022228E
:108C5A009001A5E0FFEFB402211279AB400B90001E
:108C6A0090E0FF900007EFF022900007E0FFEF701E
:108C7A000EC25B9001A5E4F022229001A5E4F02245
:106DCA009001A5E0FFEF704C900084E0FFEF602394
:106DDA00900085E0FFE532D39F4013900086E0FFE4
:106DEA0090000AEFF09001A5E004F0228026C25B31
:106DFA00228021900085E0FFE532C39F5013900066
:106E0A0086E0FF90000AEFF09001A57403F022805B
:106E1A0003C25B229001A5E0FFEF64017035900088
:106E2A0085E0FFEF24FBFFE532D39F401F90000A65
:106E3A00E0FFEF6003026F2DD25B900087E0FF90C6
:106E4A00000BEFF09001A5E004F022229001A5E4E6
:106E5A00F022229001A5E0FFEF6402702E900085D7
:106E6A00E0FFEF24FBFFE532D39F400B900087E061
:106E7A00FF90000BEFF02290000BE0FFEF6003029F
:106E8A006F2DC25B9001A5E4F022229001A5E0FFDC
:106E9A00EF64037043900085E0FF7E00EF2405FF56
:106EAA00EE3400FEAD327C00C3ED9FEE6480F8EC58
:106EBA00648098501C90000AE0FFEF7066D25B90E5
:106ECA000087E0FF90000BEFF09001A5E004F022AC
:106EDA00229001A5E4F022229001A5E0FFEF6404CC
:106EEA00703C900085E0FF7E00EF2405FFEE340041
:106EFA00FEAD327C00C3ED9FEE6480F8EC648098AE
:106F0A00500B900087E0FF90000BEFF02290000BEF
:106F1A00E0FFEF700EC25B9001A5E4F0222290011F
:046F2A00A5E4F022C8
:109B19001267708F1D9001E6E0FFEF651D600890E8
:079B290001E6E51DF0D25C2E
:019B30002212
:107CDF0090005BE0FFEF1286597D28017D32027D17
:107CEF003C037D46047D50057D5A067D64077D6EFD
:107CFF00087D78097D820A7D8C0B7D960C7DA00D09
:107D0F007DAA0E7DB40F7DBE107DC8117DD2127D70
:107D1F00DC137DE61400007DEF7BFF7A6A79F812A1
:107D2F009866227BFF7A6B7909129866227BFF7A1D
:107D3F006B791A129866227BFF7A6B792B129866F1
:107D4F00227BFF7A6B793C129866227BFF7A6B79E4
:107D5F004D129866227BFF7A6B795E129866227BB2
:107D6F00FF7A6B796F129866227BFF7A6B7980129C
:107D7F009866227BFF7A6B7991129866227BFF7A45
:107D8F006B79A2129866227BFF7A6B79B312986691
:107D9F00227BFF7A6B79C4129866227BFF7A6B790C
:107DAF00D5129866227BFF7A6B79E6129866227B52
:107DBF00FF7A6B79F7129866227BFF7A6C7908123B
:107DCF009866227BFF7A6C7919129866227BFF7A6C
:107DDF006C792A129866227BFF7A6C793B1298662F
:017DEF002271
:105601002020464C45582049562030303761202013
:1056110020002049502050524F4752414D4D494E94
:1056210047200043544353532036332E302020204B
:1056310020202043544353532036372E302020203E
:1056410020202043544353532036392E3420202028
:1056510020202043544353532037312E392020201A
:1056610020202043544353532037342E342020200C
:1056710020202043544353532037372E30202020FD
:1056810020202043544353532037392E37202020E4
:1056910020202043544353532038322E35202020DC
:1056A10020202043544353532038352E34202020CA
:1056B10020202043544353532038382E35202020B6
:1056C10020202043544353532039312E35202020AC
:1056D10020202043544353532039342E3820202096
:1056E10020202043544353532039372E3420202087
:1056F1002020204354435353203130302E3020207A
:105701002020204354435353203130332E35202061
:105711002020204354435353203130372E32202050
:105721002020204354435353203131302E3920203F
:105731002020204354435353203131342E3820202C
:105741002020204354435353203131382E38202018
:105751002020204354435353203132332E30202014
:105761002020204354435353203132372E332020FD
:105771002020204354435353203133312E382020ED
:105781002020204354435353203133362E352020DB
:105791002020204354435353203134312E332020D1
:1057A1002020204354435353203134362E322020BD
:1057B1002020204354435353203135312E342020AF
:1057C1002020204354435353203135362E37202097
:1057D1002020204354435353203135392E38202083
:1057E1002020204354435353203136322E3220207F
:1057F1002020204354435353203136352E35202069
:105801002020204354435353203136372E39202052
:105811002020204354435353203137312E3320204D
:105821002020204354435353203137332E38202036
:105831002020204354435353203137372E33202027
:105841002020204354435353203137392E3920200F
:105851002020204354435353203138332E35202008
:105861002020204354435353203138362E322020F8
:105871002020204354435353203138392E392020DE
:105881002020204354435353203139322E382020D5
:105891002020204354435353203139362E362020C3
:1058A1002020204354435353203139392E352020B1
:1058B1002020204354435353203230332E352020AF
:1058C1002020204354435353203230362E3520209C
:1058D1002020204354435353203231302E3720208F
:1058E1002020204354435353203231382E3120207D
:1058F1002020204354435353203232352E37202069
:105901002020204354435353203232392E3120205A
:105911002020204354435353203233332E3620204A
:105921002020204354435353203234312E38202039
:105931002020204354435353203235302E3320202E
:105941002020204354435353203235342E3120201C
:105951002020202020202020202020202020202046
:03596100202020E3
:1062480075840F1265BB9001E87401F09001E97440
:1062580003F07D007CFC7F1012962BE49001E8F09F
:106268009001E9F020A10875840F43E8C080067505
:10627800840F53E83F129BE87BFF7A567901129806
:1062880031129B31900003741EF0900003E070FA05
:10629800129B9590005BE0FF6005D3941440069034
:1062A800005B7401F0127CDF1288451290D01291C5
:1062B8002C12989B127975900099E0FF789F7600D0
:1062C80008A6079000A4E09001A6F0E49000EDF085
:1062D800900190F090018FF0900198F09001A0F05B
:1062E80090005274FFF0900053F0E49001E6F090B3
:1062F80001E5F0F558127987304313124A90129B42
:10630800951288451290D012912CC24380EA20A69B
:106318000E128F40E4900190F090018FF080EF30E2
:10632800461DC246124A90129B951288451290D07B
:1063380012912C129BE8E490018FF0900190F043A9
:10634800E74030580612900D1299E630A704C2A70C
:106358008002D2A71241EE123286127A9BE55BB414
:106368005514E55CB4AA0F9001E77414F09001E7A6
:10637800E070FA12797B9001A7E0704012798D5095
:106388003B127BC1127841125A48129BD812907066
:10639800129B19305C1E205D1BC25C9001E6E02454
:1063A80000FEE434179001C2F0A3CEF09001BE7451
:1063B80001F0D25DE49001F9F0026316127975904C
:1063C8000099E0FF789F760008A6079000A4E09067
:1063D80001A6F0E4900190F090018FF0900198F000
:1063E80090005BE0900052F090005374FCF012793A
:0D63F800877BFF7A567913126C4C026316F6
:108FA70001AE01C901DA01EB01FC020E0220023316
:108FB7000247025C02710287029902AB02C302DC1C
:108FC70002F50310032B03480365038403A403C5B9
:108FD70003E6040A042E04430453046A047A049142
:108FE70004A204BA04CC04E504F705100524053EE1
:108FF7000552056D0582059E05D10605061C063B33
:06900700067306AD06C76A
:109AAE00C23DC23FEF25E024A7F582E4348FF58353
:0E9ABE00E493F51A740193F51BD23ED23822C0
:09009600C23DC23FC23EC2382245
:0300A3000295289B
:10952800C0E0C0F0C083C082C0D075D000C000C009
:1095380001C002C003C004C005C006C0072058050A
:109548001281F28003129237D007D006D005D004DA
:10955800D003D002D001D000D0D0D082D083D0F0B8
:03956800D0E0321E
:03009300028E03D7
:0B8E0300C0E0C0D075D000C006C00762
:108E0E00AE84758402E5337007AFBE75BB07802F45
:108E1E00E533B40107AFBE75BB048023E533B4025E
:108E2E0007AFBE75BB068017E533B4030885BE31A8
:108E3E0075BB04800AE533B40409AFBE75BB0505E6
:108E4E00338010E533B4050885BE3275BB0480004F
:078E5E00753300C2ED8E84A4
:098E6500D007D006D0D0D0E032D5
:030083000295EEF5
:1095EE00C0E0C0F0C083C082C0D075D000C000C043
:1095FE0001C002C003C004C005C006C007C2CF121E
:10960E001CD0D007D006D005D004D003D002D00194
:0D961E00D000D0D0D082D083D0F0D0E03288
:0300730002896996
:10896900C0E0C0F0C083C082C0D075D000C000C0D4
:1089790001C002C003C004C005C006C007C2CF3091
:108989005805128ED880031291E17895E660011698
:10899900304027C240D54A05754A0A05491275D49F
:1089A900D51C09751C0A758401438820D5301B75AF
:1089B90030607584024388208010D2401277B778DE
:1089C9009616E670057604121A1A75840143881002
:1089D900758402D2ECD007D006D005D004D003D0DC
:1089E90002D001D000D0D0D082D083D0F0D0E032F4
:03006B000293D12C
:1093D100C0E0C0F0C083C082C0D075D000C000C062
:0D93E10001C002C003C004C005C006C007E3
:0E93EE008584721282C6758402C28D857284D7
:1093FC00D007D006D005D004D003D002D001D000C5
:0B940C00D0D0D082D083D0F0D0E0326E
:03005B000293838A
:10938300C0E0C0F0C083C082C0D075D000C000C0B0
:1093930001C002C003C004C005C006C00712597D46
:1093A3007897E6600116900007E0600214F0758478
:1093B30001C28DD007D006D005D004D003D002D08F
:0E93C30001D000D0D0D082D083D0F0D0E032E4
:03005300029417FD
:10941700C0E0C0F0C083C082C0D075D000C000C01B
:1094270001C002C003C004C005C006C007C28C301B
:109437005904C2598005D2591275F6D007D006D003
:1094470005D004D003D002D001D000D0D0D082D034
:0694570083D0F0D0E032EA
:03002B00020016BA
:03001600C2CF3224
:03002300029B83BA
:109B8300309904C299C262309807859956C298D217
:029B930061323D
:03001B00020019C7
:0100190032B4
:10945D00A984A2AF9264AEB1C2AF75840F53A1FEC1
:10946D008FB1E4F5849001E8E042B79001E9E04264
:10947D008F8C088D098D828C83EBF0E4F58490013F
:10948D00E9E0F4528F9001E8E0F452B78EB189848F
:04949D00A26492AF84
:0194A10022A8
:10962B00A984A2AF9264AEB1C2AF8C088D098FB181
:10963B00E4F5849001E8E0FF42B7E4F5849001E99A
:10964B00E0FD428F850982850883E4F0EDF4528FAB
:0C965B00EFF452B78EB18984A26492AF84
:0196670022E0
:109A4F00AE84A2AF9264ABB1C2AF8FB18C0A8D0B53
:0F9A5F008D828C83E493FF8BB18E84A26492AFCF
:019A6E0022D5
:100EC800202020464C45582049562020202020200C
:100ED8000020202020202020202020202049444CB1
:100EE80045002054657374696E67204D6F646520F2
:100EF80020200043726F73732042757379204D6F01
:100F08006465200053656E642049646C654D6573A3
:100F1800736167650043726F73732042757379203C
:100F28004D6F6465310043726F7373204275737936
:100F3800204D6F6465320043726F7373204275737E
:100F480079204D6F6465330043726F737320427567
:100F58007379204D6F64653400202053656E646991
:100F68006E672043574944202000205741495420A8
:100F78005544544420464C414720004C5452564F47
:100F88004950204F5554474F494E470020564F4926
:100F980050204F5554474F494E47202000202049A4
:100FA8004E434F4D494E47204C545220200020209C
:100FB800494E434F4D494E472043544353532020F5
:100FC800002020494E434F4D494E4720444353206B
:100FD800200043544353532036332E302020202002
:100FE800202043544353532036372E3020202020CE
:100FF800202043544353532036392E3420202020B8
:10100800202043544353532037312E3920202020A9
:10101800202043544353532037342E34202020209B
:10102800202043544353532037372E30202020208C
:10103800202043544353532037392E372020202073
:10104800202043544353532038322E35202020206B
:10105800202043544353532038352E342020202059
:10106800202043544353532038382E352020202045
:10107800202043544353532039312E35202020203B
:10108800202043544353532039342E382020202025
:10109800202043544353532039372E342020202016
:1010A80020204354435353203130302E3020202009
:1010B80020204354435353203130332E35202020F1
:1010C80020204354435353203130372E32202020E0
:1010D80020204354435353203131302E39202020CF
:1010E80020204354435353203131342E38202020BC
:1010F80020204354435353203131382E38202020A8
:1011080020204354435353203132332E30202020A3
:1011180020204354435353203132372E332020208C
:1011280020204354435353203133312E382020207C
:1011380020204354435353203133362E352020206A
:1011480020204354435353203134312E3320202060
:1011580020204354435353203134362E322020204C
:1011680020204354435353203135312E342020203E
:1011780020204354435353203135362E3720202026
:1011880020204354435353203135392E3820202012
:1011980020204354435353203136322E322020200E
:1011A80020204354435353203136352E35202020F8
:1011B80020204354435353203136372E39202020E2
:1011C80020204354435353203137312E33202020DD
:1011D80020204354435353203137332E38202020C6
:1011E80020204354435353203137372E33202020B7
:1011F80020204354435353203137392E392020209F
:1012080020204354435353203138332E3520202097
:1012180020204354435353203138362E3220202087
:1012280020204354435353203138392E392020206D
:1012380020204354435353203139322E3820202064
:1012480020204354435353203139362E3620202052
:1012580020204354435353203139392E3520202040
:1012680020204354435353203230332E352020203E
:1012780020204354435353203230362E352020202B
:1012880020204354435353203231302E372020201E
:1012980020204354435353203231382E312020200C
:1012A80020204354435353203232352E37202020F8
:1012B80020204354435353203232392E31202020EA
:1012C80020204354435353203233332E36202020DA
:1012D80020204354435353203234312E38202020C9
:1012E80020204354435353203235302E33202020BE
:1012F80020204354435353203235342E31202020AC
:1013080020202020202020202020202020202020D5
:1013180020204443532030303620494E5620303266
:1013280031204443532030303720494E5620323143
:1013380034204443532030313520494E562031342F
:1013480031204443532030313720494E5620303520
:1013580030204443532030323120494E562030301B
:1013680036204443532030323320494E56203034FF
:1013780037204443532030323520494E56203234EA
:1013880034204443532030323620494E56203436D8
:1013980034204443532030333120494E56203632CE
:1013A80037204443532030333220494E56203035BD
:1013B80031204443532030333620494E56203137AC
:1013C80032204443532030343320494E562034349D
:1013D80035204443532030343720494E562030328C
:1013E80033204443532030353020494E5620303185
:1013F80037204443532030353120494E562030336E
:1014080032204443532030353320494E562034355A
:1014180032204443532030353420494E562034314D
:1014280033204443532030363520494E5620323736
:1014380031204443532030373120494E5620333031
:1014480036204443532030373220494E5620323418
:1014580035204443532030373320494E5620353009
:1014680036204443532030373420494E56203137F4
:1014780034204443532031313420494E56203731EB
:1014880032204443532031313520494E56203135DE
:1014980032204443532031313620494E56203735C7
:1014A80034204443532031323220494E56203232C0
:1014B80035204443532031323520494E56203336A7
:1014C80035204443532031333120494E562033369A
:1014D80034204443532031333220494E562035348A
:1014E80036204443532031333420494E562032327B
:1014F80033204443532031343120494E5620303173
:1015080035204443532031343320494E562034315A
:1015180032204443532031343520494E5620323747
:1015280034204443532031353220494E562031313E
:1015380035204443532031353520494E5620373322
:1015480031204443532031353620494E5620323617
:1015580035204443532031363220494E5620353009
:1015680033204443532031363520494E56203235F6
:1015780031204443532031373220494E56203033EE
:1015880036204443532031373420494E56203037D3
:1015980034204443532032303520494E56203236C9
:1015A80033204443532032313220494E56203335BC
:1015B80036204443532032313420494E56203030AF
:1015C80037204443532032323320494E562031339A
:1015D80034204443532032323520494E562031328C
:1015E80032204443532032323620494E562034317B
:1015F80031204443532032343320494E562033356A
:1016080031204443532032343420494E562030325E
:1016180035204443532032343520494E5620303744
:1016280032204443532032343620494E5620353236
:1016380033204443532032353120494E5620313629
:1016480035204443532032353220494E5620343613
:1016580032204443532032353520494E5620343405
:1016680036204443532032363120494E56203733F2
:1016780032204443532032363320494E56203230EC
:1016880035204443532032363520494E56203135D3
:1016980036204443532032363620494E56203435BE
:1016A80034204443532032373120494E56203036B7
:1016B80035204443532032373420494E56203134A4
:1016C80035204443532033303620494E5620303796
:1016D80031204443532033313120494E5620363689
:1016E80034204443532033313520494E5620343278
:1016F80033204443532033323520494E5620353267
:1017080036204443532033333120494E5620343653
:1017180035204443532033333220494E5620343544
:1017280035204443532033343320494E5620353333
:1017380032204443532033343620494E5620363124
:1017480032204443532033353120494E5620323419
:1017580033204443532033353620494E5620323106
:1017680032204443532033363420494E56203133F7
:1017780031204443532033363520494E56203132E8
:1017880035204443532033373120494E56203733D0
:1017980034204443532034313120494E56203232CC
:1017A80036204443532034313220494E56203134B8
:1017B80033204443532034313320494E56203035AA
:1017C80034204443532034323320494E5620333199
:1017D80035204443532034333120494E5620373284
:1017E80033204443532034333220494E5620353178
:1017F80036204443532034343520494E5620303463
:1018080033204443532034343620494E5620323551
:1018180035204443532034353220494E5620303544
:1018280033204443532034353420494E5620323631
:1018380036204443532034353520494E562033331F
:1018480032204443532034363220494E5620323514
:1018580032204443532034363420494E5620303207
:1018680036204443532034363520494E56203333EE
:1018780031204443532034363620494E56203636DC
:1018880032204443532035303320494E56203136D8
:1018980032204443532035303620494E56203037C5
:1018A80033204443532035313620494E56203433B3
:1018B80032204443532035323320494E56203234A7
:1018C80036204443532035323620494E5620333291
:1018D80035204443532035333220494E5620333483
:1018E80033204443532035343620494E5620313373
:1018F80032204443532035363520494E5620373060
:1019080033204443532036303620494E5620363350
:1019180031204443532036313220494E5620333447
:1019280036204443532036323420494E562036332D
:1019380032204443532036323720494E5620303324
:1019480031204443532036333120494E5620363017
:1019580036204443532036333220494E56203632FF
:1019680034204443532036353420494E56203734EA
:1019780033204443532036363220494E56203436DD
:1019880036204443532036363420494E56203331CE
:1019980031204443532037303320494E56203536C2
:1019A80035204443532037313220494E56203131B7
:1019B80034204443532037323320494E56203433A1
:1019C80031204443532037333120494E5620313596
:1019D80035204443532037333220494E562032367F
:1019E80031204443532037333420494E562033376F
:1019F80031204443532037343320494E562036355E
:101A080034204443532037353420494E5620313151
:021A1800362076
:107BC1009000B3E0FFB4010A90005274FFF0E402A8
:107BD1007C8EEF64026003027C9312796F787BE6FE
:107BE1006003027C82305703027C82900197E0702F
:107BF10032D23F90009AE024FF924D90005BE0FF6B
:107C010090015BF0900098E090015CF090015DEFD5
:107C1100F012692590015EEFF012867F9001977452
:107C210002F02212839AEF64017050D23F90015802
:107C3100E0FF2442F582E43401F583E090015BF03A
:107C4100742D2FF582E43401F583E090015CF0900E
:107C51000158E090015DF012640590015EEFF09033
:107C6100015BE024D2F582E43400F583E024FF9245
:107C71004D12867F900197E014F022900197E01455
:107C8100F090005BE0900052F0900098E09000537B
:107C9100F02290018FE0B40900503D907CA3F828B8
:107CA1002873027CBE027CC1027CC4027CC7027CB8
:107CB100CA027CCD027CD0027CD3027CD60224D5C0
:107CC100028A800288D8025294024653022D06028B
:0E7CD1003CFB024EA10237EEE490018FF02240
:1024D500900190E0B40C004003022D009024E8F830
:1024E50028287302250C0225400227D70228150249
:1024F50028380228620229280229B2022A44022A1F
:1025050071022B36022C0BE49001E5F07BFF7A0E6D
:1025150079C81298317BFF7A0E79D91298669000A6
:102525005274FFF0900053F01279759000B4E0609A
:10253500031279999001907401F02220A55C12791B
:102545006F9000B4E060031279939000B1E09000C1
:1025550000F090005BE0FF900052F0900098E0FEE4
:10256500900053F09001907405F090015BEFF090AE
:10257500015CEEF090005BE090015DF01264059067
:10258500015EEFF090009AE024FF924D12867FD213
:102595003F7BFF7A0E79EA0298319001E2E064030D
:1025A500703412796F9000B4E06003127993900053
:1025B500B1E0900000F0E49001E2F09001E3E090DA
:1025C5000052F09001E4E0900053F0E4900190F0A7
:1025D50090018F0229A09001E2E0602D12796F90A1
:1025E50000B4E060031279939000B1E0900000F030
:1025F50090005BE0900052F090005374FEF0E49080
:102605000190F090018F022A40305B61304A5EC232
:102615004A90004EE0FFC39415505274D22FF582B4
:10262500E43400F583E0FFA248E4336F703FA2482D
:10263500924990004EE0900191F090004FE090019A
:1026450092F090004DE0900193F01271EC9001939F
:10265500E0641F6018900191E0FF900192E0FD7C1D
:102665000012871A90018F7402F0022D00C24A12DF
:10267500002EBF011712796F9000B4E06003127944
:10268500939000B1E0900000F0022A2E9000B5E092
:10269500602512956BEF64016006129961BF011701
:1026A5007BFF7A0E79FB129831900092E0789EF6C6
:1026B5009001907409F02212956BEF6401706830F7
:1026C5003B28C23B90019C04F0D239853E3FE53F53
:1026D50075F010A424DAF9740F35F0FA7BFF12981F
:1026E50031AF3F128D09C239802A30413AC241903B
:1026F500019EE534F075F010A4241AF9741335F031
:10270500FA7BFF12983190019EE0FF128B06900133
:102715009C7402F090018F7405F0E4900190F090A4
:102725000092E0789EF622C23BC24178A0E61846A8
:10273500703F900099E060397BFF7A0F790C129811
:1027450031900099E0FF789F760008A60790005227
:1027550074FFF0900053F012796F9000B4E06003BD
:102765001279939000B1E0900000F0900190022C56
:102775008F9000A4E0FF7003022D059001A6E06094
:1027850003022D059000A2E0FE60107003022D05E6
:102795009001A2E064016003022D059001A6EFF00F
:1027A500E49001A2F012796F9000B4E06003127911
:1027B500939000B1E0900000F090005BE090005233
:1027C500F090005374FDF0E4900190F090018F04B7
:1027D500F022900000E06003022D05305703022D22
:1027E5000590005BE0FF90015BF090015C74FFF0E9
:1027F50090015DEFF090015EF090009AE024FF9269
:102805004D12867FD23F12728E9001907403F02292
:10281500787BE66003022D05305703022D05127EF5
:10282500DC127EEB90008DE0900001F09001907439
:1028350004F022900001E06003022D0512797590E5
:1028450000B4E06003127999E4900190F09001A240
:1028550004F090005274FFF0900053F02230A5036D
:1028650002292590005BE0900052F0900098E090DE
:102875000053F012956BBF0105127981800312791F
:1028850087787BE66003022D05305703022D0590FE
:102895000197E07034D23F90009AE024FF924D906A
:1028A500005BE0FF90015BF0900098E090015CF028
:1028B50090015DEFF012692590015EEFF012867FC1
:1028C5009001977402F002728E12839AEF64017080
:1028D5004CD23F900158E0FF2442F582E43401F5E3
:1028E50083E090015BF0742D2FF582E43401F583CC
:1028F500E090015CF0900158E090015DF0126405F4
:1029050090015EEFF090015BE024D2F582E43400A3
:10291500F583E024FF924D12867F022CE4022CE41D
:10292500022D00900000E06003022D0530570302E0
:102935002D05787BE66003022D0590005274FFF0AB
:10294500900053F0128468EF64017053900158E0D1
:10295500FF2442F582E43401F583E090015BF074D5
:102965002D2FF582E43401F583E090015CF09001B0
:1029750058E090015DF0129B5C90015EEFF09001D4
:102985005BE024D2F582E43400F583E024FF924D28
:1029950012867FD23F12728E9001907407F02290BA
:1029A500008DE0900001F0900190022A40305B63B9
:1029B500304A62C24A90004EE0FFC39415505674E7
:1029C500D22FF582E43400F583E0FFA248E4336FAB
:1029D5007043A248924990004EE0900191F090001A
:1029E5004FE0900192F090004DE0900193F012714C
:1029F500EC900193E0641F601C900191E0FF900151
:102A050092E0FD7C0012871AE4900190F090018F0E
:102A1500022C8FC24A787BE66003022D05305703EE
:102A2500022D0512002EEF60079001907406F0222A
:102A350090008DE0900001F09001907408F02290D4
:102A45000001E06003022D051279759000B4E06085
:102A5500031279999001A27401F0E4900190F0902D
:102A6500005274FFF0900053F0027EEB305B633050
:102A75004A60C24A90004EE0FFC39415505474D288
:102A85002FF582E43400F583E0FFA248E4336F704C
:102A950041A248924990004EE0900191F090004F7C
:102AA500E0900192F090004DE0900193F01271ECEE
:102AB500900193E0641F601A900191E0FF900192EC
:102AC500E0FD7C0012871AE4900190F090018F02DE
:102AD5002C8FC24A789EE66003022D0590005BE0CC
:102AE500900052F090005374FDF09000B5E0FF6443
:102AF500016004EFB4021512956BBF010F900093AE
:102B0500E0900005F0900190740AF0229000B5E085
:102B1500FF64036004EFB40415129961BF010F90BF
:102B25000093E0900005F0900190740BF022022DC7
:102B35000012956BBF0108900093E0900005F0909E
:102B45000005E07003022C1F9000B5E0B401097B7D
:102B5500FF7A0F791D022C3E12796F7BFF7A0F7970
:102B65002E129866787BE66003022CF1305703023B
:102B75002CF1900197E07031D23F90009AE024FF4C
:102B8500924D90005BE0FF90015BF0900098E09023
:102B9500015CF090015DEFF012692590015EEFF0A8
:102BA50012867F900197022C8F12839AEF64017031
:102BB5004CD23F900158E0FF2442F582E43401F500
:102BC50083E090015BF0742D2FF582E43401F583E9
:102BD500E090015CF0900158E090015DF012640511
:102BE50090015EEFF090015BE024D2F582E43400C1
:102BF500F583E024FF924D12867F022CE490019725
:102C0500E014F0022CF1129961BF0108900093E0E5
:102C1500900005F0900005E070121279759000990A
:102C2500E0FF789F760008A607022D009000B5E02A
:102C3500B403097BFF7A0F793F0298667BFF7A0F11
:102C4500795012986612796F787BE66003022CF151
:102C5500305703022CF1900197E07032D23F90007B
:102C65009AE024FF924D90005BE0FF90015BF090AD
:102C75000098E090015CF090015DEFF012692590FD
:102C8500015EEFF012867F9001977402F0221283A5
:102C95009AEF64017050D23F900158E0FF2442F54D
:102CA50082E43401F583E090015BF0742D2FF58209
:102CB500E43401F583E090015CF0900158E0900167
:102CC5005DF012640590015EEFF090015BE024D2A7
:102CD500F582E43400F583E024FF924D12867F905F
:102CE5000197E014F022900197E014F090005BE06A
:102CF500900052F090005374FDF022E4900190F0A2
:012D050022AB
:108A8000129188900190E0FF700C900000E07075EA
:108A900090019004F022EF64017029205D1D900187
:108AA000C27419F0A3E4F09001BE04F0D25D90010D
:108AB0009004F07BFF7A0F796180067BFF7A0F7953
:108AC00072029866900190E0FFB402189001E5E010
:108AD00064017031F090008DE0900001F090019001
:108AE0007403F022EFB40314900001E070171279C0
:108AF000759000B4E060051279998000E490018FD0
:068B0000F0900190F0224C
:1088D800900190E0703B900068E0602B12796F90F7
:1088E80000B4E060031279939000B1E0900000F0CA
:1088F800900191E0900052F0900192E0900053F0C6
:108908009001907401F022E4900190F090018FF0B2
:1089180022900190E06401703E205D32900191E068
:10892800FE900192E07C002400FFEC3E9001C2F032
:10893800A3EFF09001BE7401F0D25D900069E09061
:10894800018F6004740480027403F0E4800E7BFFDE
:108958007A0F7972029866E490018FF0900190F096
:0189680022EC
:10529400900190E0704A900000E06003025600A282
:1052A40049924D900191E090015BF0900192E09061
:1052B400015CF090005BE090015DF01269259001C3
:1052C4005EEFF012867FD23F12728E9001977408BF
:1052D400F090008CE0900006F09001907401F022B0
:1052E400900190E06401703E127343EF60028055B8
:1052F400787BE66003025600305703025600762896
:10530400D257900197E014F0E06003025600740253
:10531400F090008CE0900006F090008EE090000C7D
:10532400F09001908069900190E064026003025360
:10533400F1127343EF6002800C90008EE0600D90D8
:10534400000CE070079001907403F022787BE66013
:1053540003025600305703025600900197E0703361
:10536400A249924D900191E090015BF0900192E08E
:1053740090015CF090005BE090015DF01269259073
:10538400015EEFF012867FD23F12728E9001977405
:1053940002F02212839AEF6401704F900158E0FFEB
:1053A4002442F582E43401F583E090015BF0742D2E
:1053B4002FF582E43401F583E090015CF09001580C
:1053C400E090015DF012640590015EEFF090015BE6
:1053D400E024D2F582E43400F583E024FF924D12F8
:1053E400867FD23F12728E0254A40254A49001907C
:1053F400E06403702E205D229001C2F0A374FFF0DC
:105404009001BE7401F0D25D127EDC127987E490C3
:105414000198F09001907404F0227BFF7A0F797266
:10542400029866900190E064047043787BE6600320
:10543400025600305703025600A249924D90019142
:10544400E090015BF0900192E090015CF090015DCE
:10545400741FF0129B5C90015EEFF012867F900146
:10546400977403F012728E9001907405F0229001EB
:1054740090E0FF64057030787BE6600302560030EC
:105484005703025600900197E0700F90008DE09052
:105494000001F09001907406F022787B7628D257B0
:1054A400900197E014F022EF640660030255E9903E
:1054B40000B5E0601F303B09304106129961EF707E
:1054C40013E490018FF0900190F0900092E0789EA8
:1054D400F60255DC305B7A304A77C24A90004EE0DF
:1054E400FFC39415506B74D22FF582E43400F58316
:1054F400E0FFA248E4336F7058A248924990004EEE
:10550400E0900191F090004FE0900192F090004DF6
:10551400E0900193F0641F6038900191E0FFC39420
:1055240015502E74D22FF582E43400F583E0FFA2E7
:1055340049E433B5071B900191E0FF900192E0FD2F
:105544007C0012871A90018F7402F0E4900190F0AD
:1055540022C24A787BE67055205752128468EF6461
:1055640001704A900158E0FF2442F582E43401F5C9
:1055740083E090015BF0742D2FF582E43401F58310
:10558400E090015CF0900158E090015DF012640538
:1055940090015EEFF090015BE024D2F582E43400E8
:1055A400F583E024FF924D12867F12728E900001E3
:1055B400E070491279759000B4E060031279999013
:1055C400005274FFF0900053F09001A27401F0E4D3
:1055D40090018FF0900190F0900099E0FF789F7611
:1055E4000008A60722900190E0D39406400EE490B0
:0D55F400018FF0900190F0789FF608F622EC
:10465300900190E070107BFF7A0F7983129831906C
:1046630001907401F022900190E064017059900070
:1046730000E06003024A8FA249924D900191E090BD
:10468300015BF0900192E090015CF090005BE090A0
:10469300015DF012692590015EEFF012867FD23F33
:1046A30012728E90008CE0900006F090008EE090E5
:1046B300000CF09000B8E09001A3F090019774070C
:1046C300F09001900247A6900190E06402703212CC
:1046D3009BD8787BE66003024A8F305703024A8FE8
:1046E3007628D257900197E014F0E06003024A8FD6
:1046F3001279819001977402F090019004F0C24AFC
:1047030022900190E064036003024804129BD820C6
:104713005B089000B8E07002803F9000B8E0FF6053
:10472300089001A3E070028030305B0D304A0A909C
:1047330001A3EFF0C24A12798112956BEF70031255
:1047430079879001E5E0B40104E402482990008EE2
:10475300E0600D90000CE070079001907404F0226B
:10476300787BE66003024A8F305703024A8F900139
:1047730097E07033A249924D900191E090015BF074
:10478300900192E090015CF090005BE090015DF09D
:1047930012692590015EEFF012867FD23F12728E6E
:1047A3009001977402F02212839AEF6401704F9084
:1047B3000158E0FF2442F582E43401F583E09001DF
:1047C3005BF0742D2FF582E43401F583E090015CF6
:1047D300F0900158E090015DF012640590015EEFE6
:1047E300F090015BE024D2F582E43400F583E02409
:1047F300FF924D12867FD23F12728E0248BA024850
:10480300BA900190E06404702E205D229001C2F002
:10481300A374FFF09001BE7401F0D25D127EDC122E
:104823007987E4900198F09001907405F0227BFF62
:104833007A0F7972029866900190E0640570467869
:104843007BE66003024A8F305703024A8FA24992E4
:104853004D900191E090015BF0900192E090015C3A
:10486300F090015D741FF0129B5C90015EEFF012FB
:10487300867F1279879001977403F012728E9001EC
:10488300907406F022900190E0FF64067030787B0C
:10489300E66003024A8F305703024A8F900197E084
:1048A300700F90008DE0900001F09001907407F07C
:1048B30022787B7628D257900197E014F022EF6498
:1048C300076003024A789000B5E0601F303B09306F
:1048D3004106129961EF7013E490018FF0900190FB
:1048E300F0900092E0789EF6024A6B12956BEF64AB
:1048F3000160030249D590008DE0900001F0204A49
:10490300030249D5C24A12956BEF64016003024961
:10491300D5900191E0FF90004EE0FEB507129000A4
:104923004FE0FF900192E0B50706E4900195F02275
:10493300EEC3941540030249D590004EE0FF24D204
:10494300F582E43400F583E0FEA248E4336E6003AD
:104953000249D5900195E0FE701BA248924990014F
:1049630094EFF090004FE0900195F090004DE090AF
:104973000196F0805D90004EE0FF6E7055A2489264
:1049830049900191EFF090004FE0900192F0900078
:104993004DE0900193F0641F6038900191E0FFC3F4
:1049A3009415502E74D22FF582E43400F583E0FF82
:1049B300A249E433B5071B900191E0FF900192E017
:1049C300FD7C0012871A90018F7402F0E49001902D
:1049D300F022787BE6706020575D128468EF6401F3
:1049E3007055900158E0FF2442F582E43401F583C9
:1049F300E090015BF0742D2FF582E43401F583E040
:104A030090015CF0900158E090015DF01264059014
:104A1300015EEFF090015BE024D2F582E43400F50F
:104A230083E024FF924D12867F9001907406F0E498
:104A330090018FF012728E900001E0703812797538
:104A43009000B4E0600312799990005274FFF090E3
:104A53000053F09001A27401F0E490018FF09001F3
:104A630090F0127EDC127EEB900099E0FF789F7647
:104A73000008A60722900190E0D39407400EE4902B
:0D4A8300018FF0900190F0789FF608F62268
:102D0600900190E06003022DEC12956BEF64017068
:102D16005B304A58C24A90004EE0FFC39415504CAF
:102D260074D22FF582E43400F583E0FFA248E43341
:102D36006F7039A248924990004EE0900191F09050
:102D4600004FE0900192F090004DE0900193F01258
:102D560071EC900193E0641F6012900191E0FF9086
:102D66000192E0FD7C0012871A023150C24A789E19
:102D7600E6600302328512956BEF6401705690008F
:102D86005EE070241279759000B4E06003127999C0
:102D96009000B5E0B4010F90005BE0900052F09017
:102DA600005374FEF022803812796F9000B4E06010
:102DB600031279931279819000B1E0900000F090AF
:102DC600005BE0900052F090005374FEF09001908A
:102DD6007401F0221279759000B4E06003127999BB
:102DE600C239E4023281900190E064017061305D85
:102DF60003022F4D90019CE0FBB4010FE53F240038
:102E0600FEE434159001C2F0A3CEF0EBB4021190AB
:102E1600019EE02400FEE434169001C2F0A3CEF039
:102E26009001BE7401F0D25D90008EE090000CF02F
:102E3600900091E0900008F0900060E0600BE49054
:102E46000190F090018F022F7590019002327590DB
:102E56000190E06402707A900000E060030232851F
:102E660090019CE064017025AF3F129AAEE53F7574
:102E7600F010A424DAF9740F35F0FA7BFF129831BA
:102E8600E53F75F010A424DAF9740F803590019CA3
:102E9600E06402600302328590019EE0FF121E5834
:102EA60090019EE075F010A4241AF9741335F0FA17
:102EB6007BFF12983190019EE075F010A4241AF958
:102EC600741335F0FA7BFF1298669001907403F044
:102ED60022900190E064037024127090EF600280EB
:102EE6001290008EE0700302328590000CE06003C1
:102EF600023285127EDC9001907404F022900190DB
:102F0600E06404704B205D3F9001C2F0A374FFF0B3
:102F16009001BE7401F0D25D127EEB127987E490C7
:102F2600019DF090005DE0600E90009FE09000092A
:102F3600F09001900232009000A0E0900002F012A2
:102F4600009690019080287BFF7A0F79720298662E
:102F5600900190E064056003023060900009E07023
:102F6600121200969000A0E0900002F0900190747A
:102F760006F02212956BEF6401706B120096303BDF
:102F860030C23B90019C7401F0853E3FC239E53F5B
:102F960075F010A424DAF9740F35F0FA7BFF129855
:102FA60031AF3F128D09E4900190F090018F02320B
:102FB60000304132C24190019EE534F075F010A414
:102FC600241AF9741335F0FA7BFF12983190019E9A
:102FD600E0FF128B0690019C7402F0E4900190F0E1
:102FE60090018F023200C23BC24112956BEF640121
:102FF6007065304A62120096C239C24A90004EE0AD
:10300600FFC39415505174D22FF582E43400F58332
:10301600E0FFA248E4336F703EA248924990004E0A
:10302600E0900191F090004FE0900192F090004DF9
:10303600E0900193F01271EC900193E0641F601729
:10304600900191E0FF900192E0FD7C0012871A90BA
:10305600018F74020230DDC24A22900190E06406BC
:103066006003023159900002E070079001907407E6
:10307600F02212956BEF64017062303B2BC23B90DD
:10308600019C04F0853E3FC239E53F75F010A4244B
:10309600DAF9740F35F0FA7BFF129831AF3F128DD3
:1030A6000990018F7405802F304131C24190019EF5
:1030B600E534F075F010A4241AF9741335F0FA7B90
:1030C600FF12983190019EE0FF128B0690019C74CE
:1030D60002F090018F7405F0E4023192C23BC241C6
:1030E60012956BEF64017068304A65120096C2391A
:1030F600C24A90004EE0FFC39415505474D22FF587
:1031060082E43400F583E0FFA248E4336F7041A205
:1031160048924990004EE0900191F090004FE09067
:103126000192F090004DE0900193F01271EC900145
:1031360093E0641F601A900191E0FF900192E0FD18
:103146007C0012871AE4900190F090018F0232758C
:10315600C24A22900190E06407600302327C90002C
:1031660001E0702D1279759000B4E0600312799930
:10317600127EEB900099E0FF789F760008A60790F4
:1031860001A27401F0C239E490018FF0900190F031
:103196002212956BEF64017065303B2CC23B9001A7
:1031A6009C04F0853E3FE53F75F010A424DAF974DF
:1031B6000F35F0FA7BFF129831AF3F128D09E4907C
:1031C6000190F090018F8032304133C24190019ED0
:1031D600E534F075F010A4241AF9741335F0FA7B6F
:1031E600FF12983190019EE0FF128B0690019C74AD
:1031F60002F0E4900190F090018F7405F022C23B3A
:10320600C24112956BEF64017069304A66120096EE
:10321600C239C24A90004EE0FFC39415505574D28D
:103226002FF582E43400F583E0FFA248E4336F70A3
:1032360042A248924990004EE0900191F090004FD2
:10324600E0900192F090004DE0900193F01271EC45
:10325600900193E0641F601B900191E0FF90019242
:10326600E0FD7C0012871AE4900190F090018F74C3
:1032760002F022C24A22E4900190F090018FF022DF
:103CFB00900190E070127BFF7A0F799412983190BB
:103D0B0001907401F0027981900190E06401706080
:103D1B00900000E060030241ED90008EE090000CFB
:103D2B00F09000B8E09001A3F090019CE0B4011278
:103D3B00AF3F129AAEE53F75F010A424DAF9740F79
:103D4B00802090019CE0640260030241ED90019E93
:103D5B00E0FF121E5890019EE075F010A4241AF992
:103D6B00741335F0FA7BFF1298669001900241DDD7
:103D7B00900190E064026003023E0B129BD8205B23
:103D8B00089000B8E07002800C9000B8E0600B90D7
:103D9B0001A3E07005127987805F305B329000B829
:103DAB00E09001A3F090019CE0B4010D303B0AE5DB
:103DBB003FB53E05C23B12798190019CE0B4020FE6
:103DCB0030410C90019EE0B53405C241127981124D
:103DDB00956BEF70031279879001E5E0B401051242
:103DEB007EDC803790008EE070030241ED90000C7A
:103DFB00E060030241ED127EDC9001907403F0222F
:103E0B00900190E0B40324205D189001C2E4F0A36C
:103E1B0074FFF09001BE7401F0D25D9001907404B8
:103E2B00F0227BFF7A0F7972029866900190E06422
:103E3B0004702C127EEB127987E490019DF09000B8
:103E4B005DE0600E90009FE0900009F09001900201
:103E5B0041359000A0E0900002F0120096801C907B
:103E6B000190E064056003023F8B900009E0701243
:103E7B001200969000A0E0900002F0900190740662
:103E8B00F02212956BEF64016003023F171200964C
:103E9B00303B39C23BE53F653E70030241ED90017B
:103EAB009C7401F0853E3FC239E53F75F010A424A8
:103EBB00DAF9740F35F0FA7BFF129831AF3F128DA0
:103ECB0009E4900190F090018F02413530413DC2E1
:103EDB004190019EE0653470030241ED90019EE537
:103EEB0034F075F010A4241AF9741335F0FA7BFF33
:103EFB0012983190019EE0FF128B0690019C740288
:103F0B00F0E4900190F090018F024135C23BC24129
:103F1B0012956BEF64017065304A62120096C239DC
:103F2B00C24A90004EE0FFC39415505174D22FF546
:103F3B0082E43400F583E0FFA248E4336F703EA2C5
:103F4B0048924990004EE0900191F090004FE09024
:103F5B000192F090004DE0900193F01271EC900102
:103F6B0093E0641F6017900191E0FF900192E0FDD8
:103F7B007C0012871A90018F7402024025C24A22DC
:103F8B00900190E0640660030240A1900002E07093
:103F9B000F90008DE0900001F09001907407F022DB
:103FAB0012956BEF64017077303B35C23BE53F6593
:103FBB003E70030241ED90019C7401F0853E3FC2BF
:103FCB0039E53F75F010A424DAF9740F35F0FA7B5C
:103FDB00FF129831AF3F128D0990018F7405803A13
:103FEB0030413CC24190019EE0653470030241EDCB
:103FFB0090019EE534F075F010A4241AF974133572
:10400B00F0FA7BFF12983190019EE0FF128B069025
:10401B00019C7402F090018F7405F0E402416BC2B5
:10402B003BC24112956BEF64017068304A65120018
:10403B0096C239C24A90004EE0FFC3941550547497
:10404B00D22FF582E43400F583E0FFA248E4336F0E
:10405B007041A248924990004EE0900191F090007F
:10406B004FE0900192F090004DE0900193F01271AF
:10407B00EC900193E0641F601A900191E0FF9001B6
:10408B0092E0FD7C0012871AE4900190F090018F72
:10409B000241DDC24A22900190E0640760030241B5
:1040AB00E412956BEF6401600302413990008DE0DF
:1040BB00900001F0303B36C23BE53F653E7003029A
:1040CB0041ED90019C7401F0853E3FE53F75F0108A
:1040DB00A424DAF9740F35F0FA7BFF129831AF3F55
:1040EB00128D09E4900190F090018F803D30413E9C
:1040FB00C24190019EE0653470030241ED90019E38
:10410B00E534F075F010A4241AF9741335F0FA7B2A
:10411B00FF12983190019EE0FF128B0690019C7468
:10412B0002F0E4900190F090018F7405F022C23BF5
:10413B00C241900001E0702D1279759000B4E060DF
:10414B0003127999127EEB900099E0FF789F76002D
:10415B0008A6079001A27401F0C239E490018FF018
:10416B00900190F02212956BEF64017069304A66F2
:10417B00120096C239C24A90004EE0FFC39415500C
:10418B005574D22FF582E43400F583E0FFA248E4A6
:10419B00336F7042A248924990004EE0900191F02B
:1041AB0090004FE0900192F090004DE0900193F061
:1041BB001271EC900193E0641F601B900191E0FF82
:1041CB00900192E0FD7C0012871AE4900190F09030
:1041DB00018F7402F022C24A22E4900190F0900108
:0341EB008FF02230
:104EA100900190E070469001E3E0900052F0900193
:104EB100E4E0900053F07BFF7A0F79A5129831E47A
:104EC1009001E2F0900052E0FF900053E0FD7C0081
:104ED10012871A900052E024D2F582E43400F5835F
:104EE100E024FF92499001907401F022900190E03A
:104EF1006401704B900000E06003025293A249925A
:104F01004D9001E3E090015BF09001E4E090015CE1
:104F1100F090005BE090015DF012692590015EEF79
:104F2100F012867FD23F12728E900082E09001A42F
:104F3100F090008EE090000CF0900190025283906E
:104F41000190E064026003025041129BD8305B1073
:104F5100304A0D900082E09001A4F0C24A1279819A
:104F610012956BEF70031279879001E5E0B4010CA3
:104F7100E4F0127EDC9001907404F0229001A4E030
:104F81007008900082E06002800C90008EE060105A
:104F910090000CE0700A127EDC9001907403F02204
:104FA100787BE660030252933057030252939001DB
:104FB10097E07032A249924D9001E3E090015BF0DD
:104FC1009001E4E090015CF090005BE090015DF005
:104FD10012692590015EEFF012867FD23F12728E28
:104FE10090019702528312839AEF6401704F9001EE
:104FF10058E0FF2442F582E43401F583E090015B3F
:10500100F0742D2FF582E43401F583E090015CF01A
:10501100900158E090015DF012640590015EEFF09F
:1050210090015BE024D2F582E43400F583E024FFB3
:10503100924D12867FD23F12728E0250EE0250EED6
:10504100900190E0B40323205D179001C2E4F0A326
:1050510074FFF09001BE7401F0D25D900190740470
:10506100F07BFF7A0F7972029866900190E06404F8
:105071007049127EEB127987787BE66003025293C6
:10508100305703025293A249924D900191E0900151
:105091005BF0900192E090015CF090015D741FF073
:1050A100129B5C90015EEFF012867F900197740372
:1050B100F012728E9001907405F022900190E0FF41
:1050C10064057030787BE660030252933057030227
:1050D1005293900197E0700F90008DE0900001F0E5
:1050E1009001907406F022787B7628D25790019730
:1050F100E014F022EF6406600302528A900001E09E
:10510100702A1279759000B4E06003127999127EC9
:10511100EB900099E0FF789F760008A6079001A226
:105121007401F0C239E490018FF0806912956BEF40
:1051310064017066303B2DC23B90019C04F0853EBA
:105141003FC239E53F75F010A424DAF9740F35F048
:10515100FA7BFF129831AF3F128D0990018F7405D0
:10516100F0E48031304133C24190019EE534F07565
:10517100F010A4241AF9741335F0FA7BFF12983158
:1051810090019EE0FF128B0690019C7402F0900149
:105191008F7405F0E4900190F022C23BC241129558
:1051A1006BEF6401600302528790008DE090000173
:1051B100F0204A03025287120096C239C24A900176
:1051C10091E0FF90004EE0FEB5071290004FE0FF26
:1051D100900192E0B50706E4900195F022EEC394A8
:1051E10015400302528790004EE0FF24D2F582E47D
:1051F1003400F583E0FEA248E4336E600302528777
:10520100900195E0FE701BA2489249900194EFF045
:1052110090004FE0900195F090004DE0900196F0E4
:10522100806490004EE0FF6E705CA248924990014C
:1052310091EFF090004FE0900192F090004DE090DE
:105241000193F01271EC900193E0641F60389001BA
:1052510091E0FFC39415502E74D22FF582E43400EF
:10526100F583E0FFA249E433B5071B900191E0FF0C
:10527100900192E0FD7C0012871AE4900190F09079
:10528100018F7402F022C24A22E4900190F0900151
:035291008FF02279
:1037EE00900190E0706390005BE0900052F09000CA
:1037FE005374FEF09001E2E0B4011D9001E4E0F597
:10380E003F7BFF7A0F79B61298319001E4E0FF12F8
:10381E008D0990019C7401F09001E2E0B4021F90BA
:10382E0001E4E090019EF07BFF7A0F79C912983186
:10383E009001E4E0FF128B0690019C7402F0E4907C
:10384E0001E2F090019004F022900190E06401708A
:10385E0058900000E06003023CFA90008EE0900069
:10386E000CF090019CE0B40112AF3F129AAEE53F0E
:10387E0075F010A424DAF9740F802090019CE06496
:10388E00026003023CFA90019EE0FF121E58900166
:10389E009EE075F010A4241AF9741335F0FA7BFF2C
:1038AE00129866900190023CEA900190E0640270DA
:1038BE0061129BD8305B2A90019CE0B4010D303B25
:1038CE000AE53FB53E05C23B12798190019CE0B4FA
:1038DE00020F30410C90019EE0B53405C2411279C1
:1038EE008112956BEF70031279879001E5E0B401B8
:1038FE0005127EDC803790008EE07003023CFA9059
:10390E00000CE06003023CFA127EDC90019074031E
:10391E00F022900190E0B40324205D189001C2E4DF
:10392E00F0A374FFF09001BE7401F0D25D9001908F
:10393E007404F0227BFF7A0F7972029866900190E0
:10394E00E064047027127EEB12798790005DE060D0
:10395E000E90009FE0900009F0900190023C75904F
:10396E0000A0E0900002F0120096801C900190E002
:10397E0064056003023A9B900009E07012120096F3
:10398E009000A0E0900002F09001907406F02212D8
:10399E00956BEF64016003023A27120096303B39B3
:1039AE00C23BE53F653E7003023CFA90019C7401F8
:1039BE00F0853E3FC239E53F75F010A424DAF97464
:1039CE000F35F0FA7BFF129831AF3F128D09E4905C
:1039DE000190F090018F023C7530413DC241900143
:1039EE009EE065347003023CFA90019EE534F0755A
:1039FE00F010A4241AF9741335F0FA7BFF129831E3
:103A0E0090019EE0FF128B0690019C7402F0E490F0
:103A1E000190F090018F023C75C23BC24112956B32
:103A2E00EF64017065304A62120096C239C24A9044
:103A3E00004EE0FFC39415505174D22FF582E4343A
:103A4E0000F583E0FFA248E4336F703EA24892492E
:103A5E0090004EE0900191F090004FE0900192F0B6
:103A6E0090004DE0900193F01271EC900193E064A0
:103A7E001F6017900191E0FF900192E0FD7C001213
:103A8E00871A90018F7402023B35C24A2290019030
:103A9E00E064066003023BB1900002E0700F9000FC
:103AAE008DE0900001F09001907407F02212956B5A
:103ABE00EF64017077303B35C23BE53F653E7003E6
:103ACE00023CFA90019C7401F0853E3FC239E53FFD
:103ADE0075F010A424DAF9740F35F0FA7BFF129802
:103AEE0031AF3F128D0990018F7405803A30413C01
:103AFE00C24190019EE065347003023CFA90019E33
:103B0E00E534F075F010A4241AF9741335F0FA7B2D
:103B1E00FF12983190019EE0FF128B0690019C746B
:103B2E0002F090018F7405F0E4023BE7C23BC24104
:103B3E0012956BEF64017068304A65120096C239B7
:103B4E00C24A90004EE0FFC39415505474D22FF524
:103B5E0082E43400F583E0FFA248E4336F7041A2A3
:103B6E0048924990004EE0900191F090004FE09005
:103B7E000192F090004DE0900193F01271EC9001E3
:103B8E0093E0641F601A900191E0FF900192E0FDB6
:103B9E007C0012871AE4900190F090018F023CEAAB
:103BAE00C24A22900190E064076003023CF190004B
:103BBE0001E0702A1279759000B4E06003127999D1
:103BCE00900099E0FF789F760008A6079001A274F6
:103BDE0001F0C239E490018FF0900190F02212951D
:103BEE006BEF64016003023C7990008DE090000160
:103BFE00F0303B36C23BE53F653E7003023CFA9027
:103C0E00019C7401F0853E3FE53F75F010A424DA67
:103C1E00F9740F35F0FA7BFF129831AF3F128D0910
:103C2E00E4900190F090018F803D30413EC2419072
:103C3E00019EE065347003023CFA90019EE534F07B
:103C4E0075F010A4241AF9741335F0FA7BFF12984C
:103C5E003190019EE0FF128B0690019C7402F0E4FD
:103C6E00900190F090018F7405F022C23BC2411278
:103C7E00956BEF64017069304A66120096C239C2C4
:103C8E004A90004EE0FFC39415505574D22FF58222
:103C9E00E43400F583E0FFA248E4336F7042A2489B
:103CAE00924990004EE0900191F090004FE090010B
:103CBE0092F090004DE0900193F01271EC90019310
:103CCE00E0641F601B900191E0FF900192E0FD7C8B
:103CDE000012871AE4900190F090018F7402F02286
:0D3CEE00C24A22E4900190F090018FF02274
:1000A600202020202020202020202020202020204A
:1000B6005245504541544552204E554D42455220D9
:1000C6002020202020202020203120746F20323054
:1000D600202053495445204E554D4245522020205C
:1000E6002020202020202020203120746F20393924
:1000F6008202001101021501148202011103041586
:1001060001632020202020202020202020202020C5
:1001160020202020202020202020202020202020D9
:10012600202020434F5552544553592042454550AF
:100136002020204354435353204F4E2048414E47DE
:10014600202020205553455220454E41424C452003
:10015600202020205245534552564520544F4E45A7
:10016600202020204E4554574F524B204D4F44459A
:100176002020204E4554574F524B204E554D424558
:100186005220202020202020202020202020202037
:100196002020202020202020202020202020202059
:1001A6002020202020202020202020202020202049
:1001B6002020202020202020202020202020202039
:1001C6002020202020202020202020202020313DFB
:1001D600454E2020202020202020202020204D4F6A
:1001E6004445202020202020202020202020544F5D
:1001F6004E4564010011020C150001640200110352
:100206000C15000164040011040C150001640800BB
:1002160011050C15000164100011060D150002C829
:10022600030111070A190101202020202020202087
:1002360020202020202020202020202020202020B8
:10024600202020202020202020434F555254455363
:100256005920424545502020204354435353204FB4
:100266004E2048414E4720202020555345522045D8
:100276004E41424C4520202020205245534552569F
:100286004520544F4E45202020204E4554574F526E
:100296004B204D4F44452020204E4554574F524B3E
:1002A600204E554D4245522020202020202020203F
:1002B6002020202020202020202020202020202038
:1002C6002020202020202020202020202020202028
:1002D6002020202020202020202020202020202018
:1002E6002020202020202020202020202020202008
:1002F60020202020313D454E202020202020202077
:10030600202020204D4F4445202020202020202042
:1003160020202020544F4E4564010011020C150088
:100326000164020011030C15000164040011040CA1
:1003360015000164080011050C1500016410001178
:10034600060D150001C8030111070A190101202035
:100356002020202020202020202020202020202097
:100366002020202020202020202020202020204364
:100376004F55525445535920424545502020202080
:100386005553455220454E41424C4520202020439E
:10039600524F535320544F4E45204D4F4445204312
:1003A600544353532F4443532043524F5353202017
:1003B6004E4554574F524B204D4F44452020204E1A
:1003C6004554574F524B204E554D42455220202002
:1003D6002020202020202020202020202020202017
:1003E60020202020202020202020313D454E202086
:1003F600202020202020202020204D4F4445202052
:1004060020202020202020202020544F4E45202030
:1004160020202020202020202020202020206401B1
:1004260000110209150001640200110309150001FB
:1004360064040011060A150001C8030111070C190E
:1004460001012020202020202020202020202020E4
:100456002020202020202020202020202020202096
:10046600202001010101010101010100000000003D
:100476000000000000000000000000000000000076
:100486000000000000000000000000000000000066
:100496000000000000000000000000000000000056
:1004A6000000000000000000000000000000000046
:1004B60000000000000000000000000020202020B6
:1004C6002020202020202020202020202020202026
:1004D6002020202020202020202020200101010192
:1004E6000101010101000000000000000000000001
:1004F60000000000000000000000000000000000F6
:1005060000000000000000000000000000000000E5
:1005160000000000000000000000000000000000D5
:1005260000000000000000000000000000000000C5
:100536000000000000002020202020202020202075
:1005460020202020202020202020202020202020A5
:1005560020202020202001010101010101010120AC
:100566002020202020202020202020202020202085
:100576002020202020202020202020202020202075
:1005860054454C434F2050524F4752414D20202056
:10059600524144494F2050524F4752414D2020204E
:1005A60050484F4E452050524F4752414D20202033
:1005B600434F4D50552050524F4752414D20202019
:1005C6002041434345535320434F44452020204474
:1005D600544D462054454C434F204C4556454C44BB
:1005E600544D4620524144494F204C4556454C42B5
:1005F60045455020524144494F204C4556454C42B2
:100606004545502054454C434F204C4556454C4398
:1006160057494420524144494F204C4556454C5673
:100626004F49434520524144494F204C45564C566C
:100636004F4943452054454C434F204C45564C505A
:1006460041474520524144494F204C4556454C436D
:100656005443535320524144494F204C45564C4431
:10066600435320524144494F204C4556454C204C5B
:10067600545220524144494F204C4556454C205235
:10068600505420524144494F204C4556454C205425
:10069600454C434F20524144494F204C45564C52FD
:1006A6004144494F2054454C434F204C45564C52EB
:1006B6004144494F204C494D4954204C45564C2005
:1006C600434F53204F5220535155454C4348202009
:1006D60020434F5320504F4C4152495459202043F8
:1006E6004F53205452494747455220564F4C544386
:1006F6004F5320414351554953542054494D454386
:100706004F532052454C454153452054494D4520B1
:1007160053454E534520504F4C415249545920534E
:10072600454E205452494747455220564F4C545344
:10073600454E20414351554953542054494D455344
:10074600454E2052454C454153452054494D452080
:100756004C545220484F4C442044454C415920505B
:100766005454205455524E4F46462054494D4552F6
:10077600455045415445522054494D454F55542006
:1007860020414E54492D4B45524348554E4B20204F
:1007960020535155454C4348205441494C20202074
:1007A60043544353532F44435320484F4C44204310
:1007B600524F535320425553592044454C415943B7
:1007C600524F5353204255535920484F4C442020F2
:1007D600204C54522053594E432042495420202045
:1007E600414456414E43454420204C4F434B202024
:1007F60020202020202020202020202020202020F3
:1008060020202020202020202020202020202020E2
:1008160020202020202020202020202020202020D2
:1008260020202020202020202020202020202020C2
:100836002020202020202020202020313D454E2031
:1008460020202020202020202020524154494F20C3
:1008560020202020202020202020303D434F5320E0
:1008660020202020202020202020313D504F5320C2
:10087600202020202020202020202031204D532001
:10088600202020202020202020203130204D5320E1
:10089600202020202020202020313030204D5320C1
:1008A60020202020202020202020202053454320C7
:1008B600202020202020202020313D534B4950204D
:1008C6002020202020202020202020202020202022
:1008D6002020202020202020202020202020202012
:1008E6005052494F52495459204C4556454C2020A8
:1008F6004C545220454E434F444520504F4C2020E7
:100906004C5452204445434F444520504F4C2020E0
:10091600205445535420494420434F444520204900
:10092600444C45204D45535341474520544D522094
:100936002020204152454120424954202020202099
:100946004D4153544552204F5220534C4156452059
:1009560044435320454E434F444520504F4C20209E
:10096600444353204445434F444520504F4C202098
:10097600434F5552544553592044454C4159202024
:10098600202048414E472054494D452020202043F1
:100996004152524945522044524F5020444C59200E
:1009A600204143434553532044454C41592020534D
:1009B600544154494F4E204944204D4F4445202030
:1009C600564F494345204F52204357494420202043
:1009D60020494420494E54455256414C202020205F
:1009E6002020435749442053504545442020202089
:1009F60043574944204652455155454E43592020B8
:100A06002043574944204D45535341474520202014
:100A16005455524E5F4F4E2044454C41592020209C
:100A26005455524E5F4F46462044454C415920206E
:100A360042454550204652455155454E4359205250
:100A4600455045415445522044495341424C452066
:100A56004155582052454C4159204D4F4445202080
:100A660043524F53532042555359204D4F4445202E
:100A76005245504541544552204741494E20202079
:100A86002054454C434F204741494E202020204EBC
:100A96004554574F524B2048414E4754494D4520E7
:100AA6002020202020202020204C4556454C202068
:100AB600202020202020202020303D4E4F524D2047
:100AC6002020202020202020202020434F44452085
:100AD6002020202020202020202020415245412077
:100AE60020202020202020303D4D415354455220C7
:100AF600202020202020202020202031204D53207F
:100B0600202020202020202020203130204D53205E
:100B1600202020202020202020313030204D53203E
:100B26002020202020202020203130205345432023
:100B36002020202020202020202031204D494E201A
:100B460020202020202020202020204D4F444520FA
:100B56002020202020202020303D564F494345208C
:100B660020202020202020202020204652455120D1
:100B76002020202020202020202020313D454E20EE
:100B860020414C41524D20434F554E5420202020A9
:100B9600524553544F524520434F554E5420202022
:100BA6002020494E54455256414C202020202020DA
:100BB6004E4554574F524B20434F44452020204921
:100BC6004E544552434F4E4E454354204D4F444E8E
:100BD6004554574F524B20494E414354495645823E
:100BE600010011022D15000182010111032D1500CE
:100BF6000182010211042D15000182010311052D48
:100C060015000178060411060119010182030A1173
:100C1600072E1500FF82030B11082E1500FF820315
:100C26000C11092E1500FF82030D110A2E1500FF67
:100C360082030E110B2E1500FF82030F110C2E15C9
:100C460000FF820310110D2E1500FF820311110EF5
:100C56002E1500FF820312110F2E1500FF820313BB
:100C660011102E1500FF82031411112E1500FF829C
:100C7600031511122E1500FF82031611132E1500EF
:100C8600FF82031711142E1500FF82031811152E6B
:100C96001500FF82011911162F15000182011A1184
:100CA600173015000182031B11182E1500FF820252
:100CB6001C11193115006382021D111A32150063C9
:100CC60082011E111B3015000182031F111C2E15F7
:100CD60000FF820220111D31150063820221111EC0
:100CE60032150063820222111F3315026382032329
:100CF6001120321501FF8203241121341502FF82CF
:100D060002251122331500638202261123321500B3
:100D160063820227112433150363820228112532C8
:100D26001500638203291126331500FA82012A1160
:100D3600273515000182012B11385415010982014E
:100D46002C11395515000182012D113A5515000156
:100D560082032E113B561501FA82032F113C5C15B6
:100D660000FF820130113D57150001820131113E0D
:100D760058150001820132113F55160001820133D8
:100D860011405515000182023411415A1500638243
:100D9600023511425B15006382023611435A150073
:100DA6006382023711445A15006382013811455E89
:100DB60015000182013911465F15000182023A11C0
:100DC600475D15006382023B114859150463820290
:100DD6003C114960150114BE0A3D114A5611000026
:100DE600820247114B5A150063820248114D601565
:100DF6000114820149114E5E15000282014A114F0B
:100E06006115000182014B11505E15000482014CF0
:100E160011515415010982014D11525415010982CF
:100E2600024E11533415006382014F116201150001
:100E36000982015011630115000982025111645D96
:100E4600150163C803521165011501018201541190
:100E5600665E1500028203551167341500FF010115
:100E66000200000200000200000000000001010173
:100E76003132333435361432320532FFFFFF191959
:100E8600196464C8FF000180000A0180000A1E1A66
:100E9600B400001E1E1E0001000002010001000039
:100EA6000A1E630A000100050520202020202020BC
:100EB6002020200A050000000101140000010000A6
:020EC60000002A
:109831008B738A7489757F01127EC2E49000E7F010
:109841009000E7E0FFC39410501AAB73AA74A97596
:109851008F827583001285F2FF127E939000E7E0FC
:0598610004F080DC2290
:106C4C008B738A7489759001F9E0B41100400302CA
:106C5C006DC9906C65F8282873026C98026CA002C0
:106C6C006CB0026CC3026CD6026CE9026CFC026D57
:106C7C000F026D22026D35026D47026D59026D6B6C
:106C8C00026D7D026D8F026DA1026DB37F01127ECC
:106C9C00C2026DC3AB73AA74A9751285D9FF127E9B
:106CAC0093026DC3AB73AA74A9759000011285F29F
:106CBC00FF127E93026DC3AB73AA74A97590000288
:106CCC001285F2FF127E93026DC3AB73AA74A97581
:106CDC009000031285F2FF127E93026DC3AB73AA70
:106CEC0074A9759000041285F2FF127E93026DC395
:106CFC00AB73AA74A9759000051285F2FF127E93EE
:106D0C00026DC3AB73AA74A9759000061285F2FFCD
:106D1C00127E93026DC3AB73AA74A975900007120F
:106D2C0085F2FF127E93026DC3AB73AA74A97590A2
:106D3C0000081285F2FF127E93807CAB73AA74A9B3
:106D4C00759000091285F2FF127E93806AAB73AACC
:106D5C0074A97590000A1285F2FF127E938058ABCD
:106D6C0073AA74A97590000B1285F2FF127E9380A2
:106D7C0046AB73AA74A97590000C1285F2FF127EB3
:106D8C00938034AB73AA74A97590000D1285F2FF31
:106D9C00127E938022AB73AA74A97590000E128593
:106DAC00F2FF127E938010AB73AA74A97590000F3A
:0E6DBC001285F2FF127E939001F9E004F0229E
:109866008B738A7489757F11127EC2E49000E7F0CB
:109876009000E7E0FFC39410501AAB73AA74A97561
:109886008F827583001285F2FF127E939000E7E0C7
:0598960004F080DC225B
:104A9000E49001A8F0A3F09001AAF09000EBF0A33D
:104AA000F09000ECE02400F582E43404F583E4F0B7
:104AB0009000ECE004F070069000EBE004F0900051
:104AC000EBE07004A3E0648070D7E49000E7F0901E
:104AD00000E7E0FFC394024003024B61EF900E64D5
:104AE00093FF9001AAE0FE04F074002EF582E434F6
:104AF00004F583EFF09001AAE06480705B9001A858
:104B0000E0FEA3E07807C333CE33CED8F9FF7C04B0
:104B10007D0012752FE49000EBF0A3F09000ECE024
:104B20002400F582E43404F583E4F09000ECE00422
:104B3000F070069000EBE004F09000EBE07004A34E
:104B4000E0648070D7E49001AAF09001A9E004F03D
:104B500070069001A8E004F09000E7E004F0024A3B
:104B6000CFE49000EAF0E49000E8F0A3F0E49000D5
:104B7000E7F09000E7E0FFC394034003024C04EF2A
:104B8000900E6693FF9001AAE0FE04F074002EF5EB
:104B900082E43404F583EFF09001AAE06480705B56
:104BA0009001A8E0FEA3E07807C333CE33CED8F956
:104BB000FF7C047D0012752FE49000EBF0A3F090D1
:104BC00000ECE02400F582E43404F583E4F0900086
:104BD000ECE004F070069000EBE004F09000EBE0F5
:104BE0007004A3E0648070D7E49001AAF09001A95A
:104BF000E004F070069001A8E004F09000E7E00403
:104C0000F0024B729000E9E004F070069000E8E0DA
:104C100004F0C39000E9E094339000E8E094005081
:104C200003024B6D9000EAE004F0E0C394145003DB
:104C3000024B66E49000EAF0E49000E8F0A3F0E4B0
:104C40009000E7F09000E7E0FFC394034003024CBC
:104C5000D6EF900E6993FF9001AAE0FE04F0740075
:104C60002EF582E43404F583EFF09001AAE064802D
:104C7000705B9001A8E0FEA3E07807C333CE33CE8B
:104C8000D8F9FF7C047D0012752FE49000EBF0A3AF
:104C9000F09000ECE02400F582E43404F583E4F0C5
:104CA0009000ECE004F070069000EBE004F090005F
:104CB000EBE07004A3E0648070D7E49001AAF09068
:104CC00001A9E004F070069001A8E004F09000E76C
:104CD000E004F0024C449000E9E004F0700690001B
:104CE000E8E004F0C39000E9E094709000E8E094FC
:104CF000005003024C3F9000EAE004F0E0C394143B
:104D00005003024C38E49000E8F0A3F0E49000E790
:104D1000F09000E7E0FFC394034003024DA3EF903F
:104D20000E6C93FF9001AAE0FE04F074002EF58251
:104D3000E43404F583EFF09001AAE06480705B90A6
:104D400001A8E0FEA3E07807C333CE33CED8F9FF45
:104D50007C047D0012752FE49000EBF0A3F090002E
:104D6000ECE02400F582E43404F583E4F09000ECF8
:104D7000E004F070069000EBE004F09000EBE070CF
:104D800004A3E0648070D7E49001AAF09001A9E048
:104D900004F070069001A8E004F09000E7E004F051
:104DA000024D119000E9E004F070069000E8E00484
:104DB000F0C39000E9E094889000E8E09413500379
:104DC000024D0C8000E49000E8F0A3F0E49000E7CE
:104DD000F09000E7E0FFC394564003024E63EF906B
:104DE0000E7293FF9001AAE0FE04F074002EF5828B
:104DF000E43404F583EFF09001AAE06480705B90E6
:104E000001A8E0FEA3E07807C333CE33CED8F9FF84
:104E10007C047D0012752FE49000EBF0A3F090006D
:104E2000ECE02400F582E43404F583E4F09000EC37
:104E3000E004F070069000EBE004F09000EBE0700E
:104E400004A3E0648070D7E49001AAF09001A9E087
:104E500004F070069001A8E004F09000E7E004F090
:104E6000024DD19000E9E004F070069000E8E00403
:104E7000F0C39000E9E094149000E8E0940050033F
:104E8000024DCC9001A8E0FEA3E07807C333CE33F7
:104E9000CED8F9FF7C047D0012752F127EDC027ED5
:014EA000EB26
:109B9500E4900059F0A3F0FFFE1274D890005BEF3B
:029BA500F022AC
:1088450075530175540075556AE49001F6F0A3F06F
:108855009001F6E0FAA3E0FBC39456EA9400504079
:1088650090005BE075F056A42478FFE5F03460CF06
:108875002BCF3AFE900059F0A3EFF01274D8AB530A
:108885000555E555AA547002055414F9EF12861FD3
:108895009001F7E004F070B89001F6E004F080B0C4
:1088A50090009BE07004D2588002C258900097E077
:1088B50024FF924F900096E024FF924490009DE0A3
:1088C50024FF924E90009CE024FF924590007CE0AE
:0288D500F52D7F
:0188D700227E
:1090D0007553017554007555BFE49001F6F0A3F087
:1090E0009001F6E0FEA3E0FFC39414EE9400503B21
:1090F0007C007D56128631EF24F9FFEE3460FE903D
:109100000059F0A3EFF01274D8AB530555E555AAFA
:10911000547002055414F9EF12861F9001F7E00411
:0B912000F070BD9001F6E004F080B597
:01912B002221
:10912C007553017554007555D3E49001F6F0A3F016
:10913C009001F6E0FEA3E0FFC39414EE9400503BC4
:10914C007C007D56128631EF24FEFFEE3460FE90DB
:10915C000059F0A3EFF01274D8AB530555E555AA9E
:10916C00547002055414F9EF12861F9001F7E004B5
:0B917C00F070BD9001F6E004F080B53B
:0191870022C5
:108D09008F73E49000E7F09000E7E0FBC394035011
:108D19003E90005BE075F099A42469FDE5F034FF0D
:108D2900FCE57375F003A42DFFE5F03CFEEB7C0038
:108D39002FFFEC3EFE1274D89000E7E02461F58223
:108D4900E43400F583EFF09000E7E004F080B89098
:108D59000061E0FE540190005CF0EE540290005D69
:108D6900F0900061E0540490005EF0EE5408900029
:0D8D79005FF0900061E05410900060F02267
:108B06008F73E49000E7F09000E7E0FBC394035016
:108B16004490005BE0FF7E007C017D50128631EFC1
:108B260024A6FDEE340AFCE57375F003A42DFFE5DB
:108B3600F03CFEEB7C002FFFEC3EFE1274D890005A
:108B4600E7E02461F582E43400F583EFF09000E776
:108B5600E004F080B2900061E0FE540190005CF009
:108B6600EE540290005DF0900061E0540490005EC7
:108B7600F0EE540890005FF0900061E05410900011
:038B860060F0227A
:06871A008F738C748D7555
:10872000E49001F6F0A3F0E57524FFFFE57434FF53
:10873000FE7C007D03128631AA06AB07AE73E5739B
:1087400025E0CE75F0EEA4FFE5F02EFEEF2448FF05
:10875000EE3423CF2BCF3AFE9001F7E02FFF9001AC
:10876000F6E03EFE1274D89001F7E02461F582E451
:108770003400F583EFF09001F7E004F0700690010B
:10878000F6E004F0C39001F7E094039001F6E09462
:10879000004094900061E0FE5401900067F0EE54B8
:0F87A00002900068F0900061E05404900069F0CE
:0187AF0022A7
:109A6F002020202020534C4156452020202020200C
:109A7F0020202020204D41535445522020202020CB
:0E9BE800127DF0127EDC127EEB7F01027EC247
:10989B009000037414F0127EDC900003E070FA90D9
:1098AB00009BE07BFF60067A9A796F80047A9A7945
:1098BB007F1298669000037414F0127EDC90000304
:0498CB00E070FA222D
:10771000C0D0C0E0C0F0C000A88475840FE5585404
:1077200007B4000D85E8F0A2F09220A2F19221802A
:1077300076B4010D85E8F0A2F09222A2F1922380A6
:1077400066B4020D85E8F0A2F09224A2F1922580A1
:1077500056B4030D85E8F0A2F09226A2F19227809C
:1077600046B4040D85E8F0A2F09218A2F1921980B7
:1077700036B4050D85E8F0A2F0921AA2F1921B80B2
:1077800026B4060D85E8F0A2F0921CA2F1921D80AD
:107790001685E8F0A2F0921EA2F1921F7558FF859F
:1077A000231E85241FD260055875590A8884D0008D
:1077B000D0F0D0E0D0D032205F0122D2B7E55A54C9
:1077C00007B4000AA22F92F7A22E92F6805EB401AF
:1077D0000AA22D92F7A22C92F68051B4020AA22B93
:1077E00092F7A22A92F68044B4030AA22992F7A241
:1077F0002892F68037B4040AA23792F7A23692F69E
:10780000802AB4050AA23592F7A23492F6801DB4FC
:10781000060AA23392F7A23292F68010B40721A290
:107820003192F7A23092F6C25F755AFF055A7584FD
:107830000F85E8E0A2F692E6A2F792E7F5E8C2B774
:017840002225
:109070009001D2E0FFEF128659909E0090A20190DD
:10908000A60290AA0390AE0490B20590B60690BADC
:109090000790BE0890C20990C60A000090CA128EBE
:1090A0006E221287B02212928C22128D862212809A
:1090B000F92212852922127EFA2212966822129330
:1090C0003322125E9822126071229001D2E4F022C3
:108E6E003061669001D3E4F0C261E5561286598EE8
:108E7E009C478EA3488EAA498EB14A8EB84B8EBFA0
:108E8E004C8EC64D8ECD4E8ED14F00008ED790019A
:108E9E00D27401F0229001D27402F0229001D274A9
:108EAE0003F0229001D27404F0229001D27405F0E6
:108EBE00229001D27406F0229001D27407F0221291
:0A8ECE009B31229001D27408F022BB
:1087B0009001D3E0FFEF70189001DA7401F090019E
:1087C000DB7401F09001D27409F09001D3E4F0223F
:1087D0009001D3E0FFEFB401189001DA7401F0903A
:1087E00001DB7402F09001D2740AF09001D3E4F03E
:1087F000229001D3E0FFEF640270499001D8E4F0C9
:10880000A3E4F09001D8E475F001128643AFF0FEC6
:10881000EF4E60269001D4E475F001128643AFF06C
:10882000FE9001D8E0FCA3E0FD74002DF5827408F1
:108830003CF583E0FD12749780C97F011200869099
:0588400001D2E4F0226A
:10928C009001D3E0FFEF70189001DA7402F09001B6
:10929C00DB7401F09001D27409F09001D3E4F02258
:1092AC009001D3E0FFEFB401189001DA7402F09052
:1092BC0001DB7402F09001D2740AF09001D3E4F057
:1092CC00229001D3E0FFEFB4020A7F0112008690D6
:0592DC0001D2E4F022C4
:108D86009001D3E0FFEF70189001DA7403F09001C0
:108D9600DB7401F09001D27409F09001D3E4F02263
:108DA6009001D3E0FFEFB401189001DA7403F0905C
:108DB60001DB7402F09001D27409F09001D3E4F063
:108DC600229001D3E0FFEFB4021C205F2F9001D464
:108DD600E0FEA3E0FF9001C2EEF0A3EFF0D25F90B9
:108DE60001D3E004F0229001D3E0FFEFB4030D209D
:0D8DF6005F0A7F011200869001D2E4F02296
:1080F9009001D3E0FFEF70189001DA7404F0900159
:10810900DB7401F09001D27409F09001D3E4F022FC
:108119009001D3E0FFEF640170749001D6E0FEA3F3
:10812900E0FF9001D8EEF0A3EFF09001E0E4F0A3B6
:10813900E4F09001D8E4F0A3E4F09001D8E475F0FC
:1081490001128643AFF0FEEF4E602B9001D4E47527
:10815900F001128643AFF0FE1274D89001E0E47585
:10816900F001128643ADF0FC74002DF58274083CD1
:10817900F583EFF080C4900800E0FF1200869001BB
:10818900E0E4F0A37401F09001D3E004F02290013F
:10819900D3E0FFEF6402703F30624D9001E0E47577
:1081A900F001128643AFF0FE74002FF58274083E89
:1081B900F583E0FF1200869001D6E0FEA3E0FF9070
:1081C90001E0E0FCA3E0FDC3ED9FEC9E50022222FA
:1081D9009001D3E004F0229001D3E0FFEFB403084B
:0981E9003062059001D2E4F0229D
:108529009001D3E0FFEF70189001DA7405F0900123
:10853900DB7401F09001D27409F09001D3E4F022C8
:108549009001D3E0FFEFB4012C9001D6E0FEA3E047
:10855900FF128C8A900800E0FF1200869001D67401
:1085690004F0A3E4F09001E0E4F0A37401F09001B9
:10857900D3E004F0229001D3E0FFEF6402703F30B2
:10858900624D9001E0E475F001128643AFF0FE748C
:10859900002FF58274083EF583E0FF1200869001F2
:1085A900D6E0FEA3E0FF9001E0E0FCA3E0FDC3ED0F
:1085B9009FEC9E500222229001D3E004F022900108
:1085C900D3E0FFEFB403083062059001D2E4F02252
:107EFA009001D3E0FFEF70189001DA7406F0900158
:107F0A00DB7401F09001D27409F09001D3E4F022FD
:107F1A009001D3E0FFEFB401289001C27430F0A3BE
:107F2A00E4F09001D4E0FEA3E0FF9001C4EEF0A3D8
:107F3A00EFF09001BE7402F0D25F9001D3E004F03A
:107F4A00229001D3E0FFEFB4020D305F03027FFB02
:107F5A009001D3E004F0229001D3E0FFEFB4030DC7
:107F6A00205E03027FFB9001D3E004F0229001D34C
:107F7A00E0FFEFB40421900800E0FF1200869001B0
:107F8A00D67404F0A3E4F09001E0E4F0A37401F0E5
:107F9A009001D3E004F0229001D3E0FFEF64057072
:107FAA003F30624D9001E0E475F001128643AFF074
:107FBA00FE74002FF58274083EF583E0FF120086F6
:107FCA009001D6E0FEA3E0FF9001E0E0FCA3E0FD13
:107FDA00C3ED9FEC9E500222229001D3E004F022CE
:107FEA009001D3E0FFEFB406083062059001D2E4B5
:027FFA00F02273
:109668009001D3E0FFEF7011C2619001D47402F051
:10967800A3E4F09001D3E004F09001D3E0FFEFB44D
:10968800011A205D179001D4E0FEA3E0FF9001C20B
:0D969800EEF0A3EFF0D25D9001D2E4F022DD
:109333009001D3E0FFEF7024306144C2619001D407
:109343007401F0A3E4F0AF567E009001D5E02FF056
:109353009001D4E03EF09001D3E004F09001D3E01B
:10936300FFEFB4011A205D179001D4E0FEA3E0FFE4
:109373009001C2EEF0A3EFF0D25D9001D2E4F022AF
:105E9800206103026070C2619001D3E0FFEF7016C9
:105EA800AF561289F97E009001D4EEF0A3EFF0907E
:105EB80001D3E004F0229001D3E0FFEFB401389061
:105EC80001D4E0FEA3E0FFEFC4F8540FC868FFEE6A
:105ED800C454F048FE9001D4EEF0A3EFF0AF561290
:105EE80089F97E009001D5E02FF09001D4E03EF0D2
:105EF8009001D3E004F0229001D3E0FFEFB4023820
:105F08009001D4E0FEA3E0FFEFC4F8540FC868FF87
:105F1800EEC454F048FE9001D4EEF0A3EFF0AF5673
:105F28001289F97E009001D5E02FF09001D4E03E6F
:105F3800F09001D3E004F0229001D3E0FFEFB40326
:105F4800389001D4E0FEA3E0FFEFC4F8540FC8680E
:105F5800FFEEC454F048FE9001D4EEF0A3EFF0AF8A
:105F6800561289F97E009001D5E02FF09001D4E017
:105F78003EF09001D3E004F0229001D3E0FFEFB4AB
:105F88000416AF561289F97E009001D6EEF0A3EF01
:105F9800F09001D3E004F0229001D3E0FFEFB405C4
:105FA800389001D6E0FEA3E0FFEFC4F8540FC868AC
:105FB800FFEEC454F048FE9001D6EEF0A3EFF0AF28
:105FC800561289F97E009001D7E02FF09001D6E0B3
:105FD8003EF09001D3E004F0229001D3E0FFEFB44B
:105FE80006389001D6E0FEA3E0FFEFC4F8540FC8CE
:105FF80068FFEEC454F048FE9001D6EEF0A3EFF02F
:10600800AF561289F97E009001D7E02FF09001D6A3
:10601800E03EF09001D3E004F0229001D3E0FFEFDE
:10602800B407459001D6E0FEA3E0FFEFC4F8540F93
:10603800C868FFEEC454F048FE9001D6EEF0A3EF16
:10604800F0AF561289F97E009001D7E02FF0900149
:10605800D6E03EF09001DBE0FF9001D3EFF0900135
:09606800DAE0FF9001D2EFF02212
:106071009001D3E0FFEF70279001E0E4F0A3E4F09A
:106081009001D6E0FEA3E0FF9001D8EEF0A3EFF07F
:106091009001DEE4F0A3E4F09001D3E004F02220CB
:1060A10061030262479001D3E0FFEFB4010EAF56E6
:1060B1001289F98F7A9001D3E004F0229001D3E0A4
:1060C100FFEF6402706CE57AC454F0F57AAF5612B2
:1060D10089F9EF257AF57A9001E0E0FEA3E0FF74FB
:1060E100002FF58274083EF583E57AF0AF7A7E00E1
:1060F1009001DFE02FF09001DEE03EF09001E1E061
:1061010004F070069001E0E004F09001D9E024FF72
:10611100F09001D8E034FFF09001D8E0FEA3E0FF59
:10612100EF4E60079001D37401F0229001D3E00497
:10613100F0229001D3E0FFEFB40316AF561289F9B4
:106141007E009001DCEEF0A3EFF09001D3E004F0CB
:10615100229001D3E0FFEFB404389001DCE0FEA30C
:10616100E0FFEFC4F8540FC868FFEEC454F048FED6
:106171009001DCEEF0A3EFF0AF561289F97E0090AA
:1061810001DDE02FF09001DCE03EF09001D3E0046E
:10619100F0229001D3E0FFEFB405389001DCE0FE7E
:1061A100A3E0FFEFC4F8540FC868FFEEC454F048F1
:1061B100FE9001DCEEF0A3EFF0AF561289F97E00FC
:1061C1009001DDE02FF09001DCE03EF09001D3E0A2
:1061D10004F0229001D3E0FFEF640670699001DCC6
:1061E100E0FEA3E0FFEFC4F8540FC868FFEEC4540B
:1061F100F048FE9001DCEEF0A3EFF0AF561289F902
:106201007E009001DDE02FF09001DCE03EF0900196
:10621100DCE0FEA3E0FF9001DEE0FCA3E0FDEDB5D4
:10622100071AECB506169001DAE0FF9001D2EFF003
:106231009001DBE0FF9001D3EFF022227F021200F8
:07624100869001D2E4F02277
:1089F9008F78E578B430037F0022E578B431037FBE
:108A09000122E578B432037F0222E578B433037F8B
:108A19000322E578B434037F0422E578B435037F73
:108A29000522E578B436037F0622E578B437037F5B
:108A39000722E578B438037F0822E578B439037F43
:108A49000922E578B441037F0A22E578B442037F1D
:108A59000B22E578B443037F0C22E578B444037F05
:108A69000D22E578B445037F0E22E578B446037FED
:078A79000F22D2637F0022EF
:0B0086008F79758400857999D2622281
:109B3100C2B5900003741EF0900003E0FFEF6004D3
:079B4100C2B580F4D2B52289
:105C980000000000000004000000080000000C00E4
:105CA80000001000000014000000180000001C0094
:105CB80000002000000024000000280000002C0044
:105CC80000003000000034000000380000003C00F4
:105CD80000004000000044000000480000004C00A4
:105CE80000005000000054000000580000005C0054
:105CF80000006000000064000000680000006C0004
:105D080000007000000074000000780000007C00B3
:105D180000108000001084000010880000108C0023
:105D280000109000001094000010980000109C00D3
:105D38000010A0000010A4000010A8000010AC0083
:105D48000010B0000010B4000010B8000010BC0033
:105D58000010C0000010C4000010C8000010CC00E3
:105D68000010D0000010D4000010D8000010DC0093
:105D78000010E0000010E4000010E8000010EC0043
:105D88000010F0000010F4000010F8000010FC00F3
:105D980000218000002184000021880000218C005F
:105DA80000219000002194000021980000219C000F
:105DB8000021A0000021A4000021A8000021AC00BF
:105DC8000021B0000021B4000021B8000021BC006F
:105DD8000021C0000021C4000021C8000021CC001F
:105DE8000021D0000021D4000021D8000021DC00CF
:105DF8000021E0000021E4000021E8000021EC007F
:105E08000021F0000021F4000021F8000021FC002E
:105E180000318000003184000031880000318C009E
:105E280000319000003194000031980000319C004E
:105E38000031A0000031A4000031A8000031AC00FE
:105E48000031B0000031B4000031B8000031BC00AE
:105E58000031C0000031C4000031C8000031CC005E
:105E68000031D0000031D4000031D8000031DC000E
:105E78000031E0000031E4000031E8000031EC00BE
:105E88000031F0000031F4000031F8000031FC006E
:1041EE009001ADE0FFEF70769001BFE0FFEFD3944A
:1041FE00034003024652206003024652C260900101
:10420E00BCE51EF0A3E51FF09001BCE0FEA3E0FFAD
:10421E00EE541FFE9001B6EEF0A3EFF09001BCE05D
:10422E00FEA3E0FFEEC4135407FF7E009001BCEE28
:10423E00F0A3EFF09001BDE0FF9001AFEFF0900121
:10424E00AEE4F09001BCE0FEA3E0FFEF4E7004D2AE
:10425E005E22229001BDE0FF9001ADEFF0229001B1
:10426E00ADE0FFEFB4011A2060030246529001B890
:10427E00E51EF0A3E51FF0C260D25E9001ADE4F042
:10428E00229001ADE0FFEF64027040206003024611
:10429E0052C2609001AEE0FFEF70119001B8E51EC2
:1042AE00F0A3E51FF09001AEE004F0229001AEE025
:1042BE00FFEF640160030246529001BAE51EF0A3BF
:1042CE00E51FF0D25E9001ADE4F0229001ADE0FF6B
:1042DE00EF640360030243FF206003024652900125
:1042EE00A7740AF0C2609001AEE0FFEF7029900152
:1042FE00B8E51EF0A3E51FF09001B4E4F0A3E4F0DE
:10430E009001B0E4F0A3E4F09001B2E4F0A3E4F085
:10431E009001AEE004F0229001AEE0FFEF64017078
:10432E00799001BCE51EF0A3E51FF09001BCE0FE04
:10433E00A3E0FF9001B1E02FF09001B0E03EF090CD
:10434E0001BCE0FCA3E0FD9001B2E475F001128621
:10435E0043AFF0FEEF25E0FFEE33FE74002FF58243
:10436E0074043EF583ECF0A3EDF09001B5E004F09B
:10437E0070069001B4E004F09001B6E0FEA3E0FFF9
:10438E009001B4E0FCA3E0FDED6F7002EC6E6003F3
:10439E000246529001AE7402F0229001AEE0FFEFA1
:1043AE00640260030246529001BAE51EF0A3E51FB7
:1043BE00F09001ADE4F09001B0E0FEA3E0FF9001BB
:1043CE00BAE0FCA3E0FDEDB5071FECB5061B9001AE
:1043DE00B6E0FEA3E0FF9001B8E0FCA3E0FD129969
:1043EE00027F007E90129B70227F017E90129B7046
:1043FE00229001ADE0FFEF640460030245302060BF
:10440E00030246529001A7740AF0C2609001AEE01A
:10441E00FFEF70299001B8E51EF0A3E51FF09001A3
:10442E00B4E4F0A3E4F09001B0E4F0A3E4F0900162
:10443E00B2E4F0A3E4F09001AEE004F0229001AEFD
:10444E00E0FFEF640170739001BCE51EF0A3E51F61
:10445E00F09001BCE0FEA3E0FF9001B1E02FF090E0
:10446E0001B0E03EF09001BCE0FCA3E0FD9001B293
:10447E00E475F001128643AFF0FEEF25E0FFEE3358
:10448E00FE74002FF58274043EF583ECF0A3EDF07C
:10449E009001B5E004F070069001B4E004F09001D4
:1044AE00B4E0FEA3E0FFEF64007003EE640260036D
:1044BE000246529001AEE004F0229001AEE0FFEF12
:1044CE0064026003024652755B559001BAE51EF018
:1044DE00A3E51FF09001B0E0FEA3E0FF9001BAE06B
:1044EE00FCA3E0FDEDB50727ECB506239001B6E081
:1044FE00FEA3E0FF127FFC7F007E90129B70900166
:10450E00B8E0FEA3E0FFEF4E6012755CAA800D7559
:10451E005B00755C007F017E90129B709001ADE494
:10452E00F0229001ADE0FFEF6405600302463D20EE
:10453E0060030246529001A7740AF0C2609001AE69
:10454E00E0FFEF70299001B8E51EF0A3E51FF09093
:10455E0001B4E4F0A3E4F09001B0E4F0A3E4F09031
:10456E0001B2E4F0A3E4F09001AEE004F022900179
:10457E00AEE0FFEF640170769001BCE51EF0A3E59E
:10458E001FF09001BCE0FEA3E0FF9001B1E02FF020
:10459E009001B0E03EF09001BCE0FCA3E0FD900184
:1045AE00B2E475F001128643AFF0FEEF25E0FFEEA8
:1045BE0033FE74002FF58274043EF583ECF0A3ED08
:1045CE00F09001B5E004F070069001B4E004F090B4
:1045DE0001B6E0FEA3E0FF9001B4E0FCA3E0FDED28
:1045EE006F7002EC6E705D9001AEE004F0229001EF
:1045FE00AEE0FFEF6402704C9001BAE51EF0A3E549
:10460E001FF09001ADE4F09001B0E0FEA3E0FF904A
:10461E0001BAE0FCA3E0FDEDB5070CECB506087F92
:10462E00007E90129B70227F017E90129B702290D2
:10463E0001ADE0FFEFD39405400A9001ADE4F09098
:05464E0001AEE4F022C2
:103286009001BFE0FFEF702A9001ADE0FFEFD3940D
:103296000240030237ED305F030237ED205D030283
:1032A60037ED9001BEE0FF9001BFEFF09001C0E462
:1032B600F0229001BFE0FFEFB401179001C2E0FEDB
:1032C600A3E0FFEE4420FE129B70C25D9001BFE4B6
:1032D600F0229001BFE0FFEF640270489001C0E069
:1032E600FFEF7019205F169001C2E0FEA3E0FFEE2B
:1032F6004440FE129B709001C0E004F0229001C091
:10330600E0FFEFB4011E305F030237ED9001C4E029
:10331600FEA3E0FF129B70C25D9001BFE4F0900136
:10332600C0E4F0229001BFE0FFEF6403706C9001EF
:10333600C0E0FFEF701C305F030237ED9001C2E082
:10334600FEA3E0FFEE4460FE129B709001C0E00415
:10335600F0229001C0E0FFEFB40118305F0302379E
:10336600ED9001C4E0FEA3E0FF129B709001C0E067
:1033760004F0229001C0E0FFEFB4021E305F0302AA
:1033860037ED9001C6E0FEA3E0FF129B70C25D9090
:1033960001BFE4F09001C0E4F0229001BFE0FFEF2E
:1033A600640460030235369001C0E0FFEF7033908D
:1033B60001C2E0FEA3E0FF9001C4E0FCA3E0FD1221
:1033C60092E19001CAE4F0A3E4F09001CCE4F0A30A
:1033D6007480F09001C8E4F0A3E4F09001C0E0042A
:1033E600F0229001C0E0FFEFB4011C305F0302370A
:1033F600ED9001C2E0FEA3E0FFEE4480FE129B705A
:103406009001C0E004F0229001C0E0FFEFB4021882
:10341600305F030237ED9001C4E0FEA3E0FF129B8C
:10342600709001C0E004F0229001C0E0FFEF640359
:103436007063305F030237ED9001C8E475F0011246
:103446008643AFF0FEEF25E0FFEE33FE74002FF566
:103456008274043EF583E0F56AA3E0F56BAF6BAECC
:103466006A129B709001CBE0256BF09001CAE035A3
:103476006AF09001CDE024FFF09001CCE034FFF03B
:103486009001CCE0FEA3E0FFEF4E60022222900105
:10349600C0E004F0229001C0E0FFEFB4041E305FEC
:1034A600030237ED9001CAE0FEA3E0FF129B709085
:1034B60001C17464F09001C0E004F0229001C0E004
:1034C600FFEF6405706A9001C1E0FFEF701990018B
:1034D600CFE004F070069001CEE004F09001BFE466
:1034E600F09001C0E4F022306046C260851E6C8513
:1034F6001F6D9001C0E4F0E56DB40011E56CB49069
:103506000C9001BFE4F09001C0E4F0C25DE56D648B
:10351600017004E56C649060030237ED9001C0E42D
:10352600F09001CFE004F070069001CEE004F022A6
:103536009001BFE0FFEF640560030237ED9001C024
:10354600E0FFEF702B9001CAE4F0A3E4F09001CC09
:103556007402F0A3E4F09001C8E4F0A3E4F0900153
:10356600C2E0FEA3E0FF128C8A9001C0E004F022C4
:103576009001C0E0FFEFB4011C305F030237ED900D
:1035860001C2E0FEA3E0FFEE44A0FE129B70900194
:10359600C0E004F0229001C0E0FFEF6402706330E7
:1035A6005F030237ED9001C8E475F001128643AF60
:1035B600F0FEEF25E0FFEE33FE74002FF582740473
:1035C6003EF583E0F56AA3E0F56BAF6BAE6A129B3E
:1035D600709001CBE0256BF09001CAE0356AF0905F
:1035E60001CDE024FFF09001CCE034FFF09001CC57
:1035F600E0FEA3E0FFEF4E600222229001C0E0044D
:10360600F0229001C0E0FFEFB4031E305F030237E3
:10361600ED9001CAE0FEA3E0FF129B709001C17419
:1036260064F09001C0E004F0229001C0E0FFEF6476
:103636000470659001C1E0FFEF70149001CFE004C3
:10364600F070069001CEE004F09001C0E4F0223064
:103656006046C260851E6C851F6D9001C0E4F0E572
:103666006DB40011E56CB4900C9001BFE4F09001CC
:10367600C0E4F0C25DE56D64017004E56C649060C1
:10368600030237ED9001CFE004F070069001CEE022
:1036960004F09001C0E4F0229001C0E0FFEF70203A
:1036A6009001CAE4F0A3E4F09001CC7402F0A3E424
:1036B600F09001C8E4F0A3E4F09001C0E004F02229
:1036C6009001C0E0FFEFB4011C305F030237ED90BC
:1036D60001C2E0FEA3E0FFEE44C0FE129B70900123
:1036E600C0E004F0229001C0E0FFEF640270633096
:1036F6005F030237ED9001C8E475F001128643AF0F
:10370600F0FEEF25E0FFEE33FE74002FF582740421
:103716003EF583E0F56AA3E0F56BAF6BAE6A129BEC
:10372600709001CBE0256BF09001CAE0356AF0900D
:1037360001CDE024FFF09001CCE034FFF09001CC05
:10374600E0FEA3E0FFEF4E600222229001C0E004FB
:10375600F0229001C0E0FFEFB4031E305F03023792
:10376600ED9001CAE0FEA3E0FF129B709001C0E05D
:1037760004F09001C17464F0229001C0E0FFEF6490
:103786000470649001C1E0FFEF70199001CFE0046E
:10379600F070069001CEE004F09001C0E4F09001D4
:1037A600BFE4F022306040C260851E6C851F6D90BC
:1037B60001C0E4F0E56DB40011E56CB4900C900125
:1037C600BFE4F09001C0E4F0C25DE56DB40118E518
:1037D6006CB490139001C0E4F09001CFE004F07057
:0737E600069001CEE004F0A3
:0137ED0022B9
:047FFC008E0F8F1045
:10800000D3E510947DE50F940040047F0180027F4A
:1080100000C3E510943FE50F940050047E018002F8
:108020007E00EE4FFFEF60030280F8E510AE0F78A0
:1080300002C333CE33CED8F9FF749A2FF582745C25
:108040003EF583E493F511740193F512E510AE0F3C
:108050007802C333CE33CED8F9FF74982FF58274EB
:108060005C3EF583E493FE740193FF8F179001AD9E
:10807000E0FFEF6405FF9001E8EFF09001AEE0FF54
:10808000EF6401FF9001E9EFF0AD12AC11AF1712F0
:10809000962B9001ADE0FFEF6405FF9001E8EFF053
:1080A0009001AEE0FFEF6403FF9001E9EFF075157A
:1080B00000751600C3E51594045033AE15AF167461
:1080C000002FF58274043EF583E0FF7E008E138F4F
:1080D00014AB14AD12AC11AF1712945D0512E5127A
:1080E000700205110516E5167002051580C690018F
:0880F000E8E4F09001E9E4F07E
:0180F8002265
:109902008E6E8F6F8C708D717B017A047900AC0240
:10991200AD01AF71AE7012752FE5712480FFE57055
:109922003400FE7B017A047980AC02AD0112752FFE
:019932002212
:048C8A008E5D8F5E0E
:108C8E00E55EAE5D7802C333CE33CED8F9FF749A6B
:108C9E002FF582745C3EF583E493F55F740193F5D2
:108CAE0060E55EAE5D7802C333CE33CED8F9FF7485
:108CBE00982FF582745C3EF583E493FE740193FF66
:108CCE008F63756100756200C3E5619404502BAD2E
:108CDE0060AC5FAF63129A4FAC61AD6274002DF55C
:108CEE008274043CF583EFF00560E5607002055F69
:0A8CFE000562E5627002056180CE98
:018D08002248
:0892E1008E648F658C668D67B9
:1092E900756800756900E5652401FFE5643400FED1
:1092F900EF25E0FFEE33FEC3E5699FE5689E50293F
:109309000567E567AE667002056614FF1274D8AC8E
:1093190068AD6974002DF58274043CF583EFF0059E
:0993290069E5697002056880BD68
:019332002218
:109B70008E188F19205FFD851825851926755A00C6
:039B8000D25F228F
:107A9B00205E03027BC09001AFE0FFEF6003027B2F
:107AAB004DC25E9001B6E0FEA3E0FFEFB4FF0BEE1C
:107ABB00B41F0775840075EF03229001B6E0FEA397
:107ACB00E0FFEEFF7E008F769001B7E0FFEF54FFF3
:107ADB00F577E576700B7FFF8F779001E57401F0FA
:107AEB0022E576B41514E577C39433500D9001E27B
:107AFB007401F09001E4E577F022E576B41614E515
:107B0B0077C39472500D9001E27402F09001E4E59A
:107B1B0077F022E576D394004028E576C394155090
:107B2B0021E577D39400401AE577C394FB5013906B
:107B3B0001E27403F09001E3E576F09001E4E57760
:107B4B00F0229001AFE0FFEF640270699001B6E0A4
:107B5B00FEA3E0FFEF64014E702B9001BFE0FFEF3F
:107B6B0070F89001C2E4F0A3747FF09001BAE0FECC
:107B7B00A3E0FF9001C4EEF0A3EFF09001BE7404FC
:107B8B00F0D25DC25E9001B6E0FEA3E0FFEF6402AF
:107B9B004E70229001BFE0FFEF70F89001BAE0FE4B
:107BAB00A3E0FF9001C2EEF0A3EFF09001BE7405CD
:057BBB00F0D25DC25E86
:017BC00022A2
:10FC0000C2AF12FCD812FD10E4F550F551E42551B5
:10FC1000FFE5503480FE12FCB6AD07AF51AE501276
:10FC2000FC5F0551E55170020550C3E550948040DA
:10FC3000DC755080755100AF51AE5012FCC7AD0756
:10FC4000AF51AE5012FC8A0551E55170020550C308
:10FC5000E55094F440E1D2AF75840075EF0122C203
:10FC6000AF75840F53A1FEE4F5B1F58443B701F5F8
:10FC700084438F018E088F098F828E83EDF0E4F527
:10FC800084538FFEF58453B7FE22C2AF75840F53A1
:10FC9000A1FE75B110E4F58443B701F584438F01EB
:10FCA0008E088F098F828E83EDF0E4F584538FFEEA
:10FCB000F58453B7FE22C2AF75B1218E0A8F0B8F28
:10FCC000828E83E493FF22C2AF75B1318E0A8F0B0F
:10FCD0008F828E83E493FF22C2AFE4FFFEE4F5B18E
:10FCE000F58443B701F584758F03AD07AC068C0826
:10FCF0008D098D828C83F0F58FF58453B7FE2FFF2D
:10FD000074043EFEC3948040D4E4F58453B7FE22CD
:10FD1000C2AF7F007E8075B110E4F58443B701F572
:04FD200084758F0354
:10FD2400AD07AC068C088D098D828C83F0F58FF5B8
:10FD34008453B7FE2FFF74043EFEC3648094744062
:08FD4400D1E4F58453B7FE225F
:0300000002007685
:0C007600787FE4F6D8FD7581A002624896
:1085D900BB010689828A83E0225002E722BBFE02A0
:0985E900E32289828A83E49322D3
:1085F200BB010CE58229F582E5833AF583E022503E
:1086020006E92582F8E622BBFE06E92582F8E22287
:0D861200E58229F582E5833AF583E49322A1
:10861F00BB010689828A83F0225002F722BBFE013A
:02862F00F32234
:10863100EF8DF0A4A8F0CF8CF0A428CE8DF0A42E5D
:02864100FE2217
:10864300A3F8E0C5F025F0F0E582158270021583EA
:06865300E0C838F0E82247
:10865900D083D082F8E4937012740193700DA3A3B0
:1086690093F8740193F5828883E4737402936860C4
:06867900EFA3A3A380DFC4
:00000001FF
